:020000040000FA
:10000000D8EF00F0FFFFFFFF04EF01F00000000059
:100010000000000000000CEF01F01000949694988E
:1000200094808B94D90E9416030E92129286939418
:10003000949C948EF3EF00F09EA8FED7AD6E000C5A
:100040009EBA02D00400FCD7AE50ABA202D0AB984F
:10005000AB881200000C050E156E15500508D8A4CB
:100060000FD00AC014F0040EE7DF0A50E5DF00EEFF
:10007000FAF0EE50141AE0DF0A2EFBD71450DCDF42
:10008000DFDF156E0608D8A4E8D7000CE40EFA6F7F
:10009000FB6B020EFC6F650EFD6F040E0A6EDBDF5C
:1000A000000CCEDF0408D8A4FCD7CADF0A6E146E99
:1000B000136E00EEFAF0C4DFEE6E141A132EFBD7A7
:1000C000BFDF141A145204E1060EB6DF04D002D0CA
:1000D000050EB2DFE6D7B8EF00F000EF01F0D6EF83
:1000E00000F0380EFA6F040EFE250A6EFEC013F003
:1000F0000900F5CFEEFF132EFBD7ADDFD6EF00F0F2
:10010000550EA76EAA0EA76EA6820000000C040E64
:100110000A5C176EEECFF5FF0D00F650070BD8A462
:1001200005D00A00840EA66EEBDF0900172EF2D769
:100130000A00840EA66EE4DF070E7EDFD6EF00F025
:10014000940EA66EDDDF400EF626E86AF722F8224E
:10015000FE2FF6D7070E70DFD6EF00F0FAC0FBF0E7
:10016000FF0EFA6F020E0A6E76DFD6EF00F099D717
:10017000FBC0F6FFFCC0F7FFFDC0F8FF00EEFEF08D
:10018000FA51B00801E1A9D7FA51340801E1A9D721
:10019000FA51320801E1BBD7FA513A0801E1D0D750
:1001A000FA51190802E172DF01D0D8D7FDEF00F053
:1001B000F86AD09EEA6AE96A810EAF6E260EAC6ECE
:1001C000900EAB6EC180C182C184C196066A076A77
:1001D000D0500F0BD0A8000ED080D082D088D88607
:1001E000D888056E1BD7D180938450DFFF0E056E33
:1001F000928693948A840400BAD7FDD70300FFFF48
:100200003BEF3FF0FFFFFFFF0B6ED8CF0CF0E0CFCE
:100210000DF00001E9CF13F0EACF0EF0E1CF0FF0BF
:10022000E2CF10F0D9CF11F0DACF12F0F3CF1AF0FD
:10023000F4CF1BF0FACF1CF000C015F001C016F08F
:1002400002C017F003C018F004C019F0F2AA2CEF96
:1002500001F0F2B43CEF02F015C000F016C001F05E
:1002600017C002F018C003F019C004F013C0E9FF72
:100270000EC0EAFF0E8E0FC0E1FF10C0E2FF11C0FA
:10028000D9FF12C0DAFF1AC0F3FF1BC0F4FF1CC075
:10029000FAFF0B500DC0E0FF0CC0D8FF1000F2CFEA
:1002A00014F0F29EF76AB80FF66E020EF7220900FC
:1002B000F55014BEF28E1200661EB01EF2CF14F07E
:1002C000F29EF76AD60FF66E020EF7220900F5507D
:1002D00014BEF28E120014256228DA331848F2CFC9
:1002E00014F0F29EF76AF80FF66E020EF72209007C
:1002F000F55014BEF28E1200E8428E445A461C4756
:10030000DC30DC30DC3032421848F2CF14F0F29EA0
:10031000F76A240FF66E030EF7220900F55014BE9B
:10032000F28E12002C52145A9A5620538A5BF2CF46
:1003300014F0F29EF76A480FF66E030EF7220900DA
:10034000F55014BEF28E1200D052D05A1A594255AE
:100350008A5BF2CF14F0F29EF76A6C0FF66E030E12
:10036000F7220900F55014BEF28E12001C218E19DE
:100370001451F2CF14F0F29EF76A8C0FF66E030E52
:10038000F7220900F55014BEF28E12003A218E19A0
:100390001451F2CF14F0F29EF76AAC0FF66E030E12
:1003A000F7220900F55014BEF28E120056218E1964
:1003B0001451F2CF14F0F29EF76ACC0FF66E030ED2
:1003C000F7220900F55014BEF28E1200BA21322233
:1003D000FA214648C848A849D84AAC4B6C4C804CD6
:1003E000FC4EA0501451F2CF14F0F29EF76A000FA9
:1003F000F66E040EF7220900F55014BEF28E1200BC
:10040000C6213E220622D848C649044B5E4C705095
:100410001451F2CF14F0F29EF76A2C0FF66E040E10
:10042000F7220900F55014BEF28E1200D2214A22A2
:1004300012229248E249424A124B344C7C4CA84C5E
:100440001650584FE64F1451F2CF14F0F29EF76A4F
:10045000620FF66E040EF7220900F55014BEF28EFC
:100460001200A864546500672C68ECCFFAFFED52C7
:10047000EFCFE8FFF96E000CD15306E081A402D063
:100480008A9401D08A8401D0F29A0400F2942CEF6D
:1004900001F09496949894808B948B928B8AD90EC9
:1004A0009416030E921292869394949C948EAEEFBF
:1004B0003FF002018A519EA8FED7AD6E0001000CEC
:1004C000020189519EA8FED7AD6E0001B7EF02F080
:1004D0009EBA05D00550061402E10400F9D7AECF4C
:1004E00098F2ABA202D0AB98AB880550061414E08A
:1004F000010E0201996F055006140EE0056A22C034
:10050000FCFF995302E1010E996F99C207F01FC0D9
:10051000FAFF1EC0E8FFF96E020198C201F0000167
:10052000000C06C088F2066A01018051070803E04A
:100530008051080806E180C18AF20001BADF43D089
:100540000101050E0201846F845106083BE08451CD
:10055000050832E1040E8A6F0001ABDF010E0201D3
:10056000876F800E866F0AC089F20001A9D70AC082
:1005700001F001C083F20201856B0A50855D18E22B
:1005800087C203F086C2E9FF87C2EAFFEFCF89F294
:1005900089C28AF200018DDF020186C2E9FF87C2AB
:1005A000EAFFEF50831B862BD8B4872B852BE5D72A
:1005B00083C28AF200017DDF00018ADF01C084F27C
:1005C0000201C2D7000188C206F0000C900E0101A2
:1005D000806F020E816F620E826F650E836F040E54
:1005E0000A6E00019EDF000C020183519EA8FED717
:1005F000AD6E0001000C02017F6B010E816F800E59
:10060000806F7F5347E1000163DF01C07CF202018C
:100610007C510408F8E106C082F2066A000158DF46
:1006200001C00AF00AC001F001C07EF202017D6B38
:100630000A507D5D1AE281C203F080C283F281C25A
:1006400084F2000145DF84C2EAFF83C2E9FF01C0F2
:10065000EFFF020180C2E9FF81C2EAFFEF507E1B7B
:10066000802BD8B4812B7D2BE3D7000131DF0150E3
:1006700002017E1B7E5308E1010E7F6F060E836F21
:100680000001B2DF05D00201050E836F0001ACDF6F
:100690000201B7D782C206F0000150EF04F081C119
:1006A0007DF2010E02017F6F820E7E6F7C6B020E67
:1006B0000A5C7C5D26E27D517D2B806F7FC203F05A
:1006C0007E517E2BD8B47F2BE96E03C0EAFFEFCFBB
:1006D00081F280C2A9FF81C2A8FFA69CA69EA68423
:1006E000F2CF00F0F29E0F01550EA76EAA0EA76E74
:1006F000A682A6B2FED7A6940050F21202017C2B6D
:10070000D6D7070E0101806F010E0A6E000109DFC6
:1007100069EF04F081C17DF2010E02017F6F820E4C
:100720007E6F82C10AF07C6B0A507C5D1AE27F51B9
:10073000036E7E517E2BD8B47F2BE96E03C0EAFF97
:100740007D517D2B826FF2CF83F2F29E82C2A9FF90
:10075000A69CA69EA680A85083BFF28EEF6E7C2B2F
:10076000E3D7E30E0101806F020E0A260001D9DEF5
:1007700069EF04F08B928B8A420E006E002EFED73A
:100780000000000C7FC202F07EC201F00232013292
:1007900002320132023201C0BEFF02320230300B9F
:1007A000006EBD50CF0B0010BD6E000CBD6A8B9467
:1007B000E1DF040E946F000C020EEA6EB60EE96ED5
:1007C000EF500EE00C0E016E006A002EFED7012ED7
:1007D000FBD7F70E006E002EFED700D0EF2EF2D71B
:1007E000000CC8DF8B940C0EBD6E9D92000E0509A7
:1007F000CA6E3B0ECB6E02017D51010A000107E07B
:10080000030A0CE0010A11E0070A16E016D0020103
:100810007F6B780E7E6F0001B5DF15D002017F6B14
:10082000270E7E6F0001AEDF0ED002017F6B350E0A
:100830007E6F0001A7DF07D0B9DF02017F6B400E9A
:100840007E6F00019FDF96DF945102017D5D0BE01A
:10085000040E7E6FAF0EB66F0001AEDF02017E2F79
:10086000F9D77DC294F0000142EF04F0400E02017E
:100870007C6F0A50020802E181C17CF27CC27DF2E9
:100880000001AFD7070E0101806F010E0A6E000153
:1008900048DE69EF04F0010E02017B6F0001ABD668
:1008A00001018051100804E1000190DE12D0010125
:1008B0008051170802E10001F2D68051180802E1C8
:1008C000000128D78051400802E10001CFD7020182
:1008D0007B6B02017BC201F00001C1EF3FF0910E82
:1008E0000101806F020E0A6E00011BDE01018151C1
:1008F00000010DE0010A10E0030A13E0010A16E00E
:10090000050A19E0010A1CE00F0A1FE023D0400E7F
:10091000AF6EA20EAC6E1FD0810EAF6EA60EAC6E87
:100920001AD0400EAF6EA60EAC6E15D02A0EAF6E6A
:10093000A60EAC6E10D0150EAF6EA60EAC6E0BD020
:10094000090EAF6EA60EAC6E06D00A0EAF6EA60EE6
:10095000AC6E01D000D0020E0201B66F00012CDF98
:10096000B5EF2EF0920E0101806F0A50410817E09A
:10097000010E816F02017D6B7D513F080EE3020E77
:100980007D25036A800FE96E010E0320EA6E7D511A
:10099000050DF3CFEFFF7D2BEFD732D00101020120
:1009A0007D6B7D513F0811E3010E7D25036A800FA9
:1009B000E96E010E0320EA6EEFCF7FF27D51050D47
:1009C000F3507F5D02E17D2BECD77D513F0802E3C0
:1009D000010E01D0000E0101816F02017D6B7D517E
:1009E0003F080EE3020E7D25036A800FE96E010EBB
:1009F0000320EA6E7D51050DF3CFEFFF7D2BEFD77E
:100A0000420E0A6E00018DDDB5EF2EF0020E0201DE
:100A1000BD5F0CE3020EEA6EBD0EE96EEF5006E01C
:100A2000020E006E002EFED7EF2EFAD70001000C4A
:100A3000950E0101806F80CF81F181CF82F182CF4D
:100A400083F1C180C192C184C196C19CC28CC28E07
:100A5000C19EC280000E016EC250C70B0110C26E53
:100A6000640E0201BD6F0001D1DFC284C2B4FED7A3
:100A7000C4CF84F10101080E016EC250C70B0110F2
:100A8000C26E640E0201BD6F0001C0DFC284C2B439
:100A9000FED7C4CF85F10101060E0A6E000141DDCB
:100AA000000C0A5007080FE1010181C192FF82C1C9
:100AB00093FF83C194FF84C189FF85C18AFF86C1EA
:100AC0008BFF0001B5DFB5EF2EF0E50E0101806F61
:100AD000070E816F020E0A6E000123DDB5EF2EF0C6
:100AE000E70E0101806FFA0E816F826B030E0A6EB2
:100AF000000117DDB5EF2EF0020180518203F3CF24
:100B000001F0F4CF00F08303F350002681518203FB
:100B1000F3500020026E00019DEF05F0000E9EBA1A
:100B2000010E016E000C7EC281F27DC280F20201D4
:100B3000836B0A0E826F0001DFD702C07EF201C014
:100B40007DF202017EC203F07D51D8B47E077D079D
:100B5000806F03C081F2805302E1815329E07F6BF3
:100B60007F51630824E3030E006E002EFED70400BD
:100B70000001D4DF015218E0010E056E8B968B98B0
:100B8000020E0201996F055006140EE0056A22C09C
:100B9000FCFF995302E1010E996F99C207F01FC043
:100BA000FAFF1EC0E8FFF96E02017F2BD9D7CAD722
:100BB0000001000C94969498070E0101806F010EBD
:100BC0000A6E0001AEDC056A010E066E8B868B880C
:100BD000010E02017E6F2C0E7D6F0001A4DF8B964B
:100BE0008B98010E02017E6F2C0E7D6F00019BDF42
:100BF000EDD7B5EF2EF05D6A080E6C6E6D6A5E6A19
:100C0000080E6E6E6F6A5F6A080E706E716A080E6B
:100C1000666E676E686E200E7A6E070E796E000C37
:100C2000010E5D6E090E6C6E6D6A010E5E6E0B0E2E
:100C30006E6E6F6A010E5F6E1F0E706E716A040E2B
:100C4000666E676E686E200E7A6E796A7AC078F08A
:100C500079C077F0000C040E5D6E090E6C6E6D6A43
:100C6000030E5E6E0B0E6E6E6F6A5F6A080E706E1C
:100C7000716A050E666E676E0D0E686E200E7A6ED6
:100C8000070E796E7AC078F079C077F0000C020E0A
:100C90005D6E090E6C6E6D6A020E5E6E0B0E6E6EF0
:100CA0006F6A020E5F6E706A716A060E666E676E1C
:100CB000686A000C030E5D6E090E6C6E6D6A020EA2
:100CC0005E6E0B0E6E6E6F6A030E5F6E706A716AF7
:100CD000080E666E676E686A4AEF0AF0050E5D6E72
:100CE000110E6C6E6D6A020E5E6E0B0E6E6E6F6A8A
:100CF000040E5F6E706A716A100E7F6E060E666E6D
:100D0000676E686A000C020E5D6E090E6C6E6D6A8D
:100D1000010E5F6E090E706E716A020E5B6E1E0E22
:100D2000666E676A686E000C050E5D6E110E6C6E65
:100D30006D6A020E5B6E020E5C6E200E7F6E050EFB
:100D4000666E676A686A72EF09F0020E5D6E090EE0
:100D50006C6E6D6A020E5B6E010E5F6E090E706E38
:100D6000716A050E666E676A686E72EF09F0050EAD
:100D70005D6E080E6C6E170E6D6E040E5E6E080EC4
:100D80006E6E170E6F6E040E5F6E706A716A200EC3
:100D90007F6E020E666E676E686A4AEF0AF0040E96
:100DA0005D6E090E6C6E170E6D6E030E5E6E0B0E91
:100DB0006E6E170E6F6E010E5F6E1F0E706E716A93
:100DC000020E666E676E080E686E4AEF0AF08B9A26
:100DD000000C8B960201A76BA7510F080DE3D8906A
:100DE000A633A53302E28B9801D08B888B86000056
:100DF0008B960000A72BF0D704000001000CBADC92
:100E0000E6DFB8DC51C0A6F250C0A5F2E2DF53C065
:100E1000A6F252C0A5F2DDDF8B98D9DF010E0201E8
:100E2000B66F0001C9DC000CEADF0201A46BA4511B
:100E300004080DE38B988B86030E006E002EFED700
:100E40008B96030E006E002EFED7A42BF0D7000168
:100E5000000C8B82000C8EDCBADFFBDF420E006ED2
:100E6000002EFED7000086DCB2DFF3DF420E006EFC
:100E7000002EFED70000000C4D520DE1555003E04E
:100E8000010A03E004D0BBDF03D0CEDF01D0E3DFF3
:100E9000010E4D6E00D0000C0201A96BA95105088E
:100EA0000DE3D890A833A73302E28B9801D08B884A
:100EB0008B8600008B960000A92BF0D7030E006EE6
:100EC000002EFED70001000C020E5D6E090E6C6E46
:100ED0006D6A020E5B6E010E5F6E090E706E716AB6
:100EE000786A776A74C07AF073C079F00A0E666E19
:100EF000676A686E96EF07F0030E726E020E646EFC
:100F000064C062F0656A65C063F0080E6A6E0E0E1A
:100F10006B6E640E696E040E586E040E596EACDF73
:100F2000060E0201A76F0001B7DFCED7000C050E39
:100F30005D6E110E6C6E6D6A020E5E6E0B0E6E6E45
:100F40006F6A040E5F6E706A716A800E7A6E796ADB
:100F5000200E7F6E080E666E676E686A48EF0AF0B4
:100F6000020E5D6E090E6C6E6D6A020E5E6E0B0EE9
:100F70006E6E6F6A050E5F6E090E706E716A74C0D8
:100F800078F073C077F0800E7A6E200E796E080EBE
:100F9000666E676E686E48EF0AF0080E806F0B0E83
:100FA000826F010E726E0F0E766EFF0E756E060E5C
:100FB0000201A76F000170DFF4EF07F0646A64C0FC
:100FC00062F0640E656E65C063F0080E6A6E0E0E08
:100FD0006B6E190E806F640E816F030E826F4F501F
:100FE000010A01E001D0D9D7030E576E4AEF0AF08B
:100FF000616A606A6B6A696A726A200E746E736AEB
:10100000766E070E756E786A776A200E7A6E796A48
:10101000010E846F8E0E836F010E866F8F0E856FAB
:10102000010E7B6E7C6A010E7D6E7E6A5490566A5C
:10103000576A586A596A5A6A5B6A5C6A4F50100A62
:10104000D8B464D0020AD8B46BD0070AD8B474D02C
:10105000040AD8B47CD0020AD8B484D0050AD8B423
:1010600090D00A0AD8B498D00B0AD8B49FD0970A67
:10107000D8B4A5D09D0AD8B4A2D0100AD8B4B4D0A0
:10108000030AD8B4C5D0160AD8B4D7D0010AD8B448
:10109000DFD0030AD8B4E6D00E0AD8B4EED0970A4F
:1010A000D8B406D1010AD8B403D1860AD8B41BD16A
:1010B0001F0AD8B42ED1180AD8B441D1040AD8B422
:1010C00046D10C0AD8B44CD1070AD8B452D18D0AF3
:1010D000D8B458D18E0AD8B45FD1070AD8B45CD13D
:1010E000160AD8B46ED1170AD8B46BD10C0AD8B48A
:1010F0007DD1030AD8B483D10C0AD8B491D18F0A18
:10110000D8B49FD1010AD8B49CD1C3D1080E646E63
:1011100064C062F0656A65C063F06A6E6CDDBAD166
:10112000080E646E64C062F0656A65C063F06A6E42
:10113000010E576E75DDAED10D0E646E64C062F0A7
:10114000656A65C063F0080E6A6E85DDA3D1040E82
:10115000646E64C062F0656A65C063F0180E6A6E02
:101160004ADD98D1020E646E64C062F0656A65C0A3
:1011700063F0180E6A6E170E6B6E010E576E50DD1F
:1011800089D1080E646E64C062F0656A65C063F060
:10119000180E6A6E60DD7ED1030E626E636A060E03
:1011A000646E656A080E6A6E72DD74D1080E646E34
:1011B00064C062F0656A65C063F06A6E7BD5080E34
:1011C000646E64C062F0656A65C063F06A6E040EA6
:1011D0007B6E030E7C6E020E576E4F50800802E14C
:1011E0007DDD01D054DD56D1030E646E64C062F023
:1011F000656A65C063F0180E6A6E0A0E6B6E640E47
:10120000696E010E7B6E7C6A020E576E40DD42D124
:10121000030E646E64C062F0656A65C063F0180E08
:101220006A6E0A0E6B6E640E696E040E7B6E030EA0
:101230007C6E020E576E2BDD2DD1140E646E64C0D1
:1012400062F0656A65C063F0080E6A6ED4DC22D174
:10125000080E646E64C062F0656A65C063F06A6E11
:10126000FADC18D1040E646E64C062F0656A65C071
:1012700063F0180E6A6EEFDC0DD1010E646E64C06F
:1012800062F0656A65C063F0080E6A6E0E0E6B6EE2
:10129000020E7B6E010E7C6E020E7D6E010E7E6E66
:1012A000020E576E040E586E040E596E2CDDF2D0ED
:1012B000050E646E64C062F0656A65C063F0080E76
:1012C0006A6E080E7B6E070E7C6E020E576E040E61
:1012D000586E040E596E180E726E4F50830801E15D
:1012E00023D533D5D7D0020E646E64C062F0656A30
:1012F00065C063F0180E6A6E170E6B6E040E7B6E7F
:10130000030E7C6E040E7D6E030E7E6E020E576E13
:101310002ED5010E646E64C062F0656A65C063F02C
:10132000180E6A6E170E6B6E040E7B6E030E7C6ECB
:10133000040E7D6E030E7E6E020E576E30D5010ECA
:10134000746E736A766EFF0E756ED6DDA3D0020ED4
:10135000746E736A030E766EFF0E756ECDDD9AD0D5
:10136000020E746E736A030E766EFF0E756EC4DD28
:1013700091D0040E746E736A070E766EFF0E756E52
:10138000BBDD88D0040E746E400E736E070E766E51
:10139000FF0E756EB1DD7ED0030E626E636A060EBF
:1013A000646E656A080E6A6E040E7B6E030E7C6EB8
:1013B000020E576E4F500F0802E190DC01D067DC3F
:1013C00069D0030E626E636A060E646E656A080E6B
:1013D0006A6E080E7B6E070E7C6E020E576E4F50C3
:1013E0001E0802E17BDC01D052DC54D0020E746E88
:1013F000736A030E766EFF0E756E7EDD4BD0080E9F
:10140000746E736A0F0E766EFF0E756E040E7B6E31
:10141000030E7C6E040E7D6E030E7E6E6DDD3AD083
:10142000020E646E64C062F0656A65C063F0180EF7
:101430006A6E0E0E6B6E640E696E020E576E63DC82
:1014400029D0800E746E736A766E070E756E0C0E60
:10145000726E0F0E846F8E0E836F0F0E866F910E5D
:10146000856F0F0E886F900E876F030E626E636A32
:10147000050E646E656A080E6A6E080E7B6E070EB6
:101480007C6E020E576E4F50850801E150D568D52D
:1014900001D094D5000C060E5D6E050E5E6E060E34
:1014A0005F6E000C070E5D6E060E5E6E070E5F6EC1
:1014B000000C010E606E616A626E636A646A640E9B
:1014C000656E050E666E676A87C268F0010E0201DE
:1014D000875D696E8AC26BF089C26AF086C257F076
:1014E000020E596E020E586E0001DCDF000C050E74
:1014F0000201866F83C288F282C287F285C28AF2B5
:1015000084C289F20001D5DF000C040E0201866F4F
:1015100083C288F282C287F285C28AF284C289F2CB
:101520000001C7DF000C080E5D6E080E5F6EF9EF5C
:101530000BF0090E5D6E090E5F6EBFEF0AF00A0E2A
:10154000606E616A626E636A646A010E656E900E17
:10155000666E676A400E686E3F0E696E84C26BF0FD
:1015600083C26AF082C257F0556AC20E516EB20E43
:10157000506E0A0E536E120E526E6F80DAD7000C48
:10158000050E0201826F846B836B0001D8DFF9EFD7
:101590000BF0040E0201826F846F836B0001CFDFBA
:1015A000F9EF0BF0010E606E616A626E636A646A45
:1015B000640E656E050E666E676A050E626E636A7E
:1015C00083C268F0010E0201835D696E6B6A400E92
:1015D0006A6E020E596E020E586E000163DF000C37
:1015E000040E576E6F8482C283F2DCDF000C050E9E
:1015F000576E82C283F2D6DF000C190E6C6E630E3A
:101600006D6E030E6E6E060E576E4F50230A03E08A
:10161000070A0CE015D0010E606E616A626E636AA3
:10162000646A050E656E666A676A0AD0606A640E4F
:10163000616E626A636E646A656A666A676A00D030
:10164000F9EF0BF0010E606E616A626E636A646AA4
:10165000050E656E666E676A080E686E070E696E27
:101660006B6A400E6A6E020E556E6F6A6F82010ED3
:10167000566E200E4F5CE10FD8B0BBD01F0F0BEFA2
:101680000CF0050E576E010E596E010E586E6F92DA
:1016900002DFAFD0050E576E020E596E020E586E65
:1016A000FADEA7D0040E576E010E596E010E586E69
:1016B0006F92F1DE9ED0040E576E020E596E020E2E
:1016C000586EE9DE96D00201836B080E826F856B3F
:1016D000200E846F00010BDF8CD00201836B080E9B
:1016E000826F856B200E846F00010FDF82D00201B4
:1016F000836B200E826F856B400E846F0001F7DED6
:1017000078D00201836B200E826F856B400E846F50
:101710000001FBDE6ED00201836B100E826F856BC1
:10172000400E846F0001E3DE64D00201836B100E73
:10173000826F856B400E846F0001E7DE5AD0020194
:10174000836B400E826F856B846F0001D0DE51D0B9
:101750000201836B400E826F856B846F0001D5DEC2
:1017600048D0020E606E616A626E636A646A780EC7
:10177000656E1E0E666E676A100E686E0F0E696EDD
:101780006B6A100E6A6E050E576ECDD6F9D601D76C
:10179000080E0201826F000123DF2BD0080E020128
:1017A000826F000124DF25D0100E0201826F00013C
:1017B00017DF1FD0100E0201826F000118DF19D051
:1017C000200E0201826F00010BDF13D0200E0201F8
:1017D000826F00010CDF0DD0400E0201826F00010C
:1017E000FFDE07D0400E0201826F000100DF01D052
:1017F00004D70201816B81517F0809E3036A81C22A
:10180000E9FF010E0324EA6EEF6A812BF4D73C90C6
:10181000000153EF0EF0F2CF14F0F29EE824F76AC5
:10182000F7363B0FF66E180EF7220A00F550FA6EE7
:101830000800F55014BEF28EF96E94169416C61672
:10184000F017F017EE163E17621782169416F2176D
:10185000A416B616F217B616B616DA1602175017F1
:1018600016178C172A1790179C17C017CC17D81764
:10187000E417A817B4178E170A0E5D6E400E6F6E30
:10188000710E6E6E070E5E6E400E716E750E706E8E
:101890000A0E5F6E400E736E7F0E726E8A6B950E2F
:1018A000896F0C0E8B6F12EF0EF00A0E5D6E400EFC
:1018B0006F6E420E6E6E020E5B6E0B0E5F6E400E12
:1018C000736E4F0E726E12EF0EF00B0E5D6E400EC9
:1018D0006F6E420E6E6E020E5B6E0C0E5F6E400EF1
:1018E000736E4F0E726E8A6BB90E896F180E8B6F06
:1018F00012EF0EF00A0E5D6E400E6F6E710E6E6E80
:10190000020E5B6E0A0E5F6E400E736E7F0E726E7D
:101910008A6BA10E896F180E8B6F12EF0EF0020109
:10192000B56BB551030812E3D890B43302E28B983B
:1019300001D08B888B86030E006E002EFED78B960F
:10194000030E006E002EFED7B52BEBD70001000C66
:101950000201B46B0001E3DF0201B36BB35117085E
:1019600014E3D890B133B033AF3302E28B9801D097
:101970008B888B86030E006E002EFED78B96030E8F
:10198000006E002EFED7B32BE9D70001000C8CA50A
:101990000ED00201B26BB16BB06BAF6B0001D8DF40
:1019A0000201B26BB16BB06BAF6B0001D1DF64C0F1
:1019B000A6F2020165C0A7F266500409A86F67C0CD
:1019C000A9F267C0B2F2B16F65C0B0F264C0AFF205
:1019D0000001BEDF64C0A6F2020165C0A7F2665036
:1019E0000409A86F67C0A9F267C0B2F2B16F65C001
:1019F000B0F264C0AFF20001ABDF0201B26BB16BB9
:101A0000B06BAF6B0001A4DF0201B26BB16BB06BC6
:101A1000AF6B00019DDF64C0A6F2020165C0A7F2B2
:101A200066500409A86F67C0A9F267C0B2F2B16F2F
:101A300065C0B0F264C0AFF200018ADF0201B26B90
:101A4000B16BB06BAF6B000183DF000C8C6B010ED0
:101A5000836F846B866B856F886B876F020E566E03
:101A6000010E5A6E010E5B6E010E5C6E400E4F5CF5
:101A7000FC0FD8B0D7D0040F17EF0EF0676A666A74
:101A8000010E656E646A400E696E080E686E400E47
:101A90006B6E010E6A6E400E6D6E050E6C6E756A91
:101AA000020E746E776A766E796A786E7B6A7A6EE9
:101AB000070E576E030E596E030E586E020E556ECA
:101AC000200E7C6E1F0E7D6E200E7E6E060E806FC9
:101AD0007F6A826B170E816F100E836F0F0E846FFB
:101AE000866B100E856F010E886F876B8C85C4D650
:101AF000676A666A020E656E646A400E696E030E5E
:101B0000686E400E6B6E010E6A6E6D6A6C6A756E61
:101B1000900E746E776A280E766E796A020E786E71
:101B20007B6A140E7A6E070E576E010E556EC20E4A
:101B3000516EB20E506E8A0E536E120E526E400EE1
:101B40007C6E3F0E7D6E7E6A806B580E7F6E826B60
:101B5000010E816F8C818C83A8D6676A666A020E3B
:101B6000656E646A400E696E686A6B6E010E6A6E1D
:101B70006D6A6C6A756E900E746E776A140E766E6E
:101B8000796A020E786E7B6A140E7A6E070E576EB3
:101B9000010E556EC20E516EB20E506E8A0E536E0D
:101BA000120E526E400E7C6E3F0E7D6E7E6A806B12
:101BB000B00E7F6E826B010E816F8C818C8385D617
:101BC000676A666A010E656E646A400E696E080E89
:101BD000686E400E6B6E010E6A6E6D6A6C6A756A95
:101BE000C80E746E776A766E796A020E786E7B6ABA
:101BF0007A6E070E576E010E556EC20E516EB20E02
:101C0000506E8A0E536E120E526E200E7C6E1F0E98
:101C10007D6E200E7E6E806B800E7F6E826B170E47
:101C2000816F68D63CEC07F0B2DE53EF0EF0F2CFD6
:101C300014F0F29EE824F76AF736530FF66E1C0E86
:101C4000F7220A00F550FA6E0800F55014BEF28E25
:101C5000F96E7C1AF01A5A1BC01B4D6A5480020E92
:101C6000556E030E566E080E576E040E586E596E62
:101C7000020E5A6E5B6E5C6E0C0E5D6E080E5E6E32
:101C80000D0E5F6E9496949894808B968B984E5020
:101C900005E0010A06E0030A05E005D0F8EC07F0CC
:101CA00002D0D0D4D3D6000E54B0010E006ED8901E
:101CB00000360050036AF2CF82F2F29E4FEC01F040
:101CC0000900F5CF03F0020182BFF28E266E03C039
:101CD00027F0D8905634036AF2CF81F2F29E0001C9
:101CE0005EEC01F00900F5CF03F0020181BFF28E36
:101CF0002A6E03C02BF0D8905734036AF2CF81F2DA
:101D0000F29E00016FEC01F00900F5CF03F0020133
:101D100081BFF28E286E03C029F0D8905834036A30
:101D2000F2CF81F2F29E000185EC01F00900F5CFBF
:101D300003F0020181BFF28E2E6E03C02FF0D89007
:101D40005934036AF2CF81F2F29E000197EC01F060
:101D50000900F5CF03F0020181BFF28E2C6E03C0A3
:101D60002DF0D8905A34036AF2CF81F2F29E00012E
:101D7000A9EC01F00900F5CF03F0020181BFF28E5A
:101D8000306E03C031F0D8905B34036AF2CF81F239
:101D9000F29E0001B9EC01F00900F5CF03F0020159
:101DA00081BFF28E326E03C033F0D8905C34036A88
:101DB000F2CF81F2F29E0001C9EC01F00900F5CFEB
:101DC00003F0020181BFF28E346E03C035F0D8906B
:101DD0005D34036AF2CF81F2F29E0001D9EC01F08A
:101DE0000900F5CF03F0020181BFF28E366E03C009
:101DF00037F0D8905E34036AF2CF81F2F29E000190
:101E0000F3EC01F00900F5CF03F0020181BFF28E7F
:101E1000386E03C039F0D8905F34036AF2CF81F294
:101E2000F29E000109EC02F00900F5CF03F0020177
:101E300081BFF28E3A6E03C03BF04D5204E10001C7
:101E40003CEC07F002010001000C020180517F0B05
:101E5000006E00384E6E4E32070E4E1680C24FF0A6
:101E60000001FBDE000C02018351050803E3036A55
:101E7000835102D0036A060E846F03C085F2EA6ABA
:101E8000830EE96E82C2E2FF81C2E1FF03C002F06D
:101E900084C201F0015202E0022A02D0025206E09E
:101EA000E6CFEEFF012EFCD7022EFAD70001000C80
:101EB000000CEA6A260EE96E7FC282F27EC281F2CF
:101EC00080C283F235EC02F0000C81C180F2BDDFEC
:101ED0000A5002080CE2020E0A5C02017D6F010E3C
:101EE0007F6F820E7E6F7DC280F20001E2DF070EFF
:101EF0000101806F010E0A6E000191EC02F0B5EF56
:101F00002EF07DC24EF07EC24FF0A7DE90EF0FF0B4
:101F100081C17DF202017F6B82C17EF20001F1D7A7
:101F20000A5003080CE2030E0A5C02017D6F010EE9
:101F30007F6F830E7E6F7DC280F20001BADF070ED5
:101F40000101806F010E0A6E000191EC02F0B5EF05
:101F50002EF0D6EC03F0070E0101806F010E0A6E21
:101F6000000191EC02F0B5EF2EF04F5002084BE16A
:101F7000A8C2ABF2A7C2AAF20201AF6BAE6BABC2B2
:101F8000B1F2AAC2B0F2AC6BAC510D080FE3D8901D
:101F9000B133B033AD6BD8B0AD2BACA103D0AD51E4
:101FA000AF1B02D0AD51AE1BAC2BEED7010EAF1B59
:101FB000AF5302E1D89001D0D880AA37AB37AE53E7
:101FC00002E1D89001D0D880AA37AB378B888B86B6
:101FD00000008B960000B26BB2510F080DE3D89051
:101FE000AB33AA3302E28B9801D08B888B8600003A
:101FF0008B960000B22BF0D78B888B8600008B96D7
:1020000000001DD000018B888B8600008B9600009D
:102010000201A96BA9510D080DE3D890A833A7338D
:1020200002E28B9801D08B888B8600008B96000093
:10203000A92BF0D78B888B8600008B960000060EAC
:10204000006E002EFED700000400000131EF10F0FA
:10205000A4C2A7F24CEC07F0A6C2A8F2A5C2A7F250
:1020600084D7000C72A015D075500201A25DD8B4BF
:1020700002D000010ED07650A35DD8B402D000018A
:1020800008D000012BEC07F076C061F075C060F05D
:1020900031D00201A351615C04E311E16050A25D03
:1020A0000EE37450A35D27E303E17350A25D23E3C5
:1020B0006150745C20E303E17350605C1CE24D6A84
:1020C0000001F8EC07F03CEC07F074500201A35D4E
:1020D00012E303E17350A25D0EE372B20CD0A46B65
:1020E0003F0EA66FFF0EA56F0001B2DF74C061F056
:1020F00073C060F002016150A35D0EE303E1A251E1
:10210000605C0AE2060EA76F00014CEC07F0602A43
:10211000D8B4612A0201EFD70001000C78C0A3F205
:1021200077C0A2F29FDF020E0201A46F3F0EA66FDE
:10213000FF0EA56F00018CDF000C0201A36BA26BE8
:10214000000190DF030E0201A46FA66BFF0EA56FC6
:1021500000017EDF000C0201A36BA26B000182DF95
:102160007AC0A3F279C0A2F27DDF000C88C2A7F288
:102170004CEC07F089C2B6F2DCEC03F0000C010E67
:102180000201A76F00014CEC07F0070E0201A76FD8
:1021900000014CEC07F07EC288F27FC289F2E6DFD4
:1021A000010E0201A76F00014CEC07F0070E0201BF
:1021B000A76F00014CEC07F0000C6CC07EF266C00B
:1021C0007FF2DDDF000C6EC07EF267C07FF2D7DFEA
:1021D000000C70C07EF268C07FF2D1DF0201A36BF9
:1021E000A26B00013FDF030E0201A46FA66BFF0E7E
:1021F000A56F00012DDFE7DF000C6CC088F266C020
:1022000089F2B4DF000C6EC088F267C089F2AEDFDD
:10221000000CF3DFF8DF000C7EC288F27FC289F287
:10222000A5DF080E0201886F020E896F00019EDF94
:10223000000C6CC07EF266C07FF2EEDF000C6EC058
:102240007EF267C07FF2E8DF000C70C088F268C0E1
:1022500089F28CDF000C0201A66B4F501F081BE1B6
:10226000A76BA7510F0816E38B86420E006E002E57
:10227000FED7000000D082B802D0D89001D0D8801C
:10228000A4C2EAFFA3C2E9FFEC52ED32ED328B9615
:10229000A72BE7D710D14F500208D8A4F7D08B86D0
:1022A00000D08B968B8600D08B968B8600D082B820
:1022B00002D0D89001D0D880A4C2EAFFA3C2E9FF1F
:1022C000EC52ED32ED328B968B8600D082B802D084
:1022D000D89001D0D880A4C2EAFFA3C2E9FFEC5293
:1022E000ED32ED328B968B8600D082B802D0D8903A
:1022F00001D0D880A4C2EAFFA3C2E9FFEC52ED32BC
:10230000ED328B968B8600D082B802D0D89001D067
:10231000D880A4C2EAFFA3C2E9FFEC52ED32ED324D
:102320008B968B8600D082B802D0D89001D0D8800E
:10233000A4C2EAFFA3C2E9FFEC52ED32ED328B9664
:102340008B8600D082B802D0D89001D0D880A4C2A9
:10235000EAFFA3C2E9FFEC52ED32ED328B968B8699
:1023600000D082B802D0D89001D0D880A4C2EAFFB1
:10237000A3C2E9FFEC52ED32ED328B968B8600D092
:1023800082B802D0D89001D0D880A4C2EAFFA3C2FC
:10239000E9FFEC52ED32ED328B968B8600D082B89D
:1023A00002D0D89001D0D880A4C2EAFFA3C2E9FF2E
:1023B000EC52ED32ED328B968B8600D082B802D093
:1023C000D89001D0D880A4C2EAFFA3C2E9FFEC52A2
:1023D000ED32ED328B968B8600D082B802D0D89049
:1023E00001D0D880A4C2EAFFA3C2E9FFEC52ED32CB
:1023F000ED328B968B8600D082B802D0D89001D077
:10240000D880A4C2EAFFA3C2E9FFEC52ED32ED325C
:102410008B968B8600D082B802D0D89001D0D8801D
:10242000A4C2EAFFA3C2E9FFEC52ED32ED328B9673
:102430008B8600D082B802D0D89001D0D880A4C2B8
:10244000EAFFA3C2E9FFEC52ED32ED328B968B86A8
:1024500000D082B802D0D89001D0D880A4C2EAFFC0
:10246000A3C2E9FFEC52ED32ED328B968B8600D0A1
:1024700082B802D0D89001D0D880A4C2EAFFA3C20B
:10248000E9FFEC52ED32ED328B9615D0A86BA851D6
:102490000F0811E38B8600D082B802D0D89001D00B
:1024A000D880A4C2EAFFA3C2E9FFEC52ED32ED32BC
:1024B0008B96A82BECD7A65302E1D89001D0D880F8
:1024C000A4C2EAFFA3C2E9FFEC52ED32ED32A3C28F
:1024D000E9FFA4C2EAFFEFCF00F0EC503F0B036E20
:1024E0000050ED52EF6E03C0ECFF060E006E002EA2
:1024F000FED700000400000188EF12F0A0C2A7F28E
:102500004CEC07F09488A2C2A4F2A1C2A3F2A3D615
:102510009498000C8AC292F289C291F20201906BE7
:102520008F51905D21E292C203F09151912BD8B46A
:10253000922B936F03C094F203C0A3F2A26F000129
:1025400091DD020190518D25936F000E8E21946FC5
:10255000040EA06F94C2A2F293C2A1F20001CEDFDA
:10256000020E02019027DCD70001000C0201BD6BB6
:10257000BD5103080EE3D890BC3302E28B9801D022
:102580008B888B8600D000008B9600D00000BD2B7E
:10259000EFD70001000C8B960201C16BC1510F08EF
:1025A0000FE3D890C033BF3302E28B9801D08B8801
:1025B0008B8600D000008B9600D00000C12BEED798
:1025C00004000001000C020E0201BB6FB60EBA6FD0
:1025D000BC6B0001CBDF020E0201BA25016E000EBA
:1025E000BB21036E01C0E9FFEA6EEFCFBCF20E0E15
:1025F000BCC2BDF2C06FBCC2BFF20001CCDF0201A1
:10260000BC6B0001B3DF6E0E0201C06FF80EBF6F2E
:102610000001C1DF0201BC6B0001A8DF010E020155
:10262000BA25016E000EBB21036E01C0E9FFEA6E00
:10263000EFCFBCF20E0EBCC2BDF2C06FBCC2BFF287
:102640000001A9DF0201BC6B000190DF6E0E0201E8
:10265000C06FF70EBF6F00019EDF0201BC6B00016F
:1026600085DFBBC203F00201BAC2E9FFBBC2EAFFC9
:10267000EFCFBCF20E0EBCC2BDF2C06FBCC2BFF247
:10268000000189DF0201BC6B000170DF6E0E0201E8
:10269000C06FF60EBF6F00017EDF000C0201B35366
:1026A00003E1B2512F080EE2B3530CE1B2513008EE
:1026B00009E305E1B15306E1B0510D0803E3B56B41
:1026C000B46B03D0100EB56FB46BBC6B00014EDF62
:1026D0008E0E0201C06FA60EBF6F00015CDF02010B
:1026E000BC6B000143DFEF0E0201C06FBF6B000146
:1026F00052DF0201BC6B000139DFF80E0201C06F2E
:10270000BF6B000148DF0201BC6B00012FDF02013B
:10271000B451A609B66FB5518C09B76FC06FB6C278
:10272000BFF2000138DFB3C2B9F2B2C2B8F2B1C22F
:10273000B7F2B0C2B6F247DF000C94888B8600D0A7
:1027400000008B968B8600D000008B968B8600D085
:1027500000008B968B8600D000008B968B8600D075
:1027600000008B968B8600D000008B968B8600D065
:1027700000008B968B8600D000008B968B8600D055
:10278000000082B802D0D89001D0D880B3C2EAFF4E
:10279000B2C2E9FFED328B968B8600D0000082B882
:1027A00002D0D89001D0D880B3C2EAFFB2C2E9FF0C
:1027B000ED328B968B8600D0000082B802D0D89084
:1027C00001D0D880B3C2EAFFB2C2E9FFED328B96E6
:1027D0008B8600D0000082B802D0D89001D0D8807B
:1027E000B3C2EAFFB2C2E9FFED328B968B8600D00E
:1027F000000082B802D0D89001D0D880B3C2EAFFDE
:10280000B2C2E9FFED328B968B8600D0000082B811
:1028100002D0D89001D0D880B3C2EAFFB2C2E9FF9B
:10282000ED328B968B8600D0000082B802D0D89013
:1028300001D0D880B3C2EAFFB2C2E9FFED328B9675
:102840008B8600D0000082B802D0D89001D0D8800A
:10285000B3C2EAFFB2C2E9FFED328B9694988B9631
:10286000000C8CC2B3F28BC2B2F28AC2B1F289C23E
:10287000B0F214DF0201906B8F51905D14E2090EEB
:10288000BC6F000173DE036A020190518D25956FC4
:102890008E510320966FB36F95C2B2F200014DDFE7
:1028A0000201902BE9D70001000C0201B96B3C0E2C
:1028B000B86FB76B060EB66F000185DE0C0E020115
:1028C000BC6F000153DE0201C06BBF6B000163DE11
:1028D000000C020E0201A86FA8A32FD0A851FF0878
:1028E0002CE0BC6B000142DE500E0201C06FA60E50
:1028F000BF6F000150DE0201BC6B000137DE6E0EBF
:102900000201C06FF50EBF6F000145DE0201BC6B16
:1029100000012CDE0201C06BBF6B00013CDE020E29
:102920000201BC6F000122DE020E0201B36FA80E8D
:10293000B26F000102DF0201CFD70001000C0201DB
:10294000BC6B000113DE840E0201C06FA60EBF6FC8
:10295000000121DE0201BC6B000108DE880E0201CD
:10296000C06FA60EBF6F000116DE0201BC6B000136
:10297000FDDD0E0E0201C06F550EBF6F00010BDEB4
:102980000201BC6B0001F2DD6E0E0201C06FA70EEA
:10299000BF6F000100DE0201BC6B0001E7DD0E0E1F
:1029A0000201C06FAA0EBF6F0001F5DD0201BC6B12
:1029B0000001DCDD6E0E0201C06FA70EBF6F0001CB
:1029C000EADD0201BC6B0001D1DD820E0201C06FA5
:1029D000A60EBF6F0001DFDD0201BC6B0001C6DD8A
:1029E0000201C06BBF6B0001D6DD6FA40BD00201EA
:1029F000BC6B0001BBDD0201C06BBF6B0001CBDD16
:102A000068DF1AD00201BC6B0001B0DD645066249F
:102A10000201A86FB66F0001DCEC03F0655067247B
:102A20000201A86FA8C2BDF2000106EC05F0020188
:102A3000C06BBF6B0001AFDD0201BC6B000196DD16
:102A4000940E0201C06FA60EBF6F0001A4DD000C42
:102A50000201A15303E1A0511F0816E2A15313E1A3
:102A6000A0512F0810E33CB00ED000011EDFA1C220
:102A7000B3F2A0C2B2F29FC2B1F29EC2B0F20EDEB9
:102A80005EDF3C80020175D09E6BF80E9F171F0E13
:102A9000A017A16BA131026EA031016E9F31006EB3
:102AA00002320132003202320132003200C0A2F2A0
:102AB000A231A36FA333A3331F0EA317A251070B99
:102AC000016E010EA26F015204E0D890A237012ED0
:102AD000FCD7036AA3C2E9FF010E0324EA6EEF509C
:102AE000A21547E1036AA3C2E9FF010E0324EA6EBF
:102AF000EF50A211EF6EA56BA46BA5533AE1A45160
:102B00001F0837E30400A76BA66BA7531DE1A6516E
:102B10003F081AE304000001C8DEA1C2B3F2A0C25C
:102B2000B2F29FC2B1F29EC2B0F2B8DD08DF6A50C5
:102B300002019E276B509F23000EA023A1236A5001
:102B4000A6276B50A723E1D7A731036EA631026EEB
:102B500003320232033202320332023203320232D1
:102B600003320232030E03160250A4270350A5239A
:102B7000C4D70001BAEF18F00201B56BB5510208D5
:102B80000EE3D890B23302E28B9801D08B888B860B
:102B900000D000008B9600D00000B52BEFD7D89066
:102BA000B23302E28B9801D08B888B86B3C2B6F227
:102BB0000001DCEC03F0B4C2BDF206EC05F000D07D
:102BC00000008B9600D0000064C0B6F2DCEC03F08D
:102BD00065C0BDF206EC05F0000C9FC2A3F29EC2D8
:102BE000A2F20201A16BA051A15D47E20F0EBC6FE2
:102BF0000001BCDCA3C203F00201A2C2E9FFA3C230
:102C0000EAFFECCFA5F2ED52EFCFA4F2A5C2C0F2DD
:102C1000A4C2BFF20001BFDC0201B26B62C0B3F21A
:102C200063C0B4F20001A8DF0201C06BBF6B0001FA
:102C3000B2DC0201B26B62C0B3F263C0B4F2000155
:102C40009BDF2A0E0201C06FF60EBF6F0001A3DCEE
:102C50000201BC6B00018ADC0201C06BBF6B00018A
:102C60009ADC0201A151010B006ED8900036005091
:102C7000A227000EA323A12BB6D70001F9EF18F06D
:102C80009FC2A2F29EC2A1F2D8900201A033A0532B
:102C9000D8B47AD0A2C203F0A1C200F0020EA127DC
:102CA000D8B0A22B00C0E9FF03C0EAFFECCF03F0CD
:102CB000ED52EFCFA3F203C0A4F26DC0A6F20D0E49
:102CC000BC6F000153DCA4C2C0F2A3C2BFF263DC3C
:102CD0000201B26B60C0B3F261C0B4F200014CDF1C
:102CE0000201C06BBF6B000156DC0C0E0201BC6F11
:102CF00000013CDCA4C2C0F2A3C2BFF24CDC020162
:102D0000B26B60C0B3F261C0B4F2000135DF020102
:102D1000C06BBF6B00013FDC0201A607D8B402D034
:102D20000001E3D70E0EBC6F000120DCA4C2C0F28C
:102D3000A3C2BFF230DC0201B26B60C0B3F261C06B
:102D4000B4F2000119DF0201C06BBF6B000123DC8C
:102D5000090E0201BC6F000109DC020E0201B36F13
:102D6000A50EB26F0001E9DC090E0201BC6F000183
:102D7000B6EC12F0020E0201B36FA50EB26F0001A5
:102D8000DCDC0201A00783D70001F9EF18F0020193
:102D9000B36BB26BB16BB06B000180DC0201AC6B4A
:102DA0006850AC5D10E20D0EBC6F0001B6EC12F085
:102DB000FF0E0201C06FBF6F0001CBEC12F0020EDC
:102DC0000201AC27EDD70001000C0201AE51010851
:102DD00061E2AF6B020EAE5DAF5D22E20D0EBC6F25
:102DE0000001B6EC12F00201ADC203F0ACC200F07B
:102DF000020EAC27D8B0AD2B00C0E9FF03C0EAFF3C
:102E0000ECCFB1F2ED52EFCFB0F2B1C2C0F2B0C22E
:102E1000BFF20001CBEC12F0020E0201AF27DAD7AD
:102E20000F0EBC6F0001B6EC12F00201ADC203F050
:102E3000ACC200F0020EAC27D8B0AD2B00C0E9FF49
:102E400003C0EAFFECCFB1F2ED52EFCFB0F2B1C266
:102E5000C0F2B0C2BFF20001CBEC12F00201B26BC3
:102E600060C0B3F261C0B4F2000186DE0201C06B43
:102E7000BF6B0001CBEC12F00D0E0201BC6F000124
:102E8000B6EC12F0FF0E0201C06FBF6F0001CBEC79
:102E900012F002010001000CA1C2ABF2A0C2AAF222
:102EA0009FC2A9F29EC2A8F202019E516914A56FA9
:102EB000A4C2A7F2A55325E0A551685CA66FA65150
:102EC000A75D02E2A7C2A6F26FA00CD000015FDFEF
:102ED000ABC2B3F2AAC2B2F2A9C2B1F2A8C2B0F2B6
:102EE0004EEC13F0A3C2ADF2A2C2ACF2A6C2AEF297
:102EF00000016BDF0201A651A75FA651A227000EB9
:102F0000A3236850A75D10E3A3C2ADF2A2C2ACF246
:102F100068C0AEF2000159DF68500201A227000E1E
:102F2000A3236850A75FEDD7A7532AE06FA01FD057
:102F300000012DDF0201A751A45D006E016A026A43
:102F4000036A0050A825AC6F0150A921AD6F025053
:102F5000AA21AE6F0350AB21AF6FB36FAEC2B2F216
:102F6000ADC2B1F2ACC2B0F200014EEC13F0A3C29C
:102F7000ADF2A2C2ACF2A7C2AEF2000126DF02019E
:102F8000000123EF19F0A1C2B1F2A0C2B0F29FC2BA
:102F9000AFF29EC2AEF2A3C2A6F2A2C2A5F2D89030
:102FA0000201A433A453D8B496D0A6C203F0A5C29C
:102FB00000F0020EA527D8B0A62B00C0E9FF03C081
:102FC000EAFFECCF03F0ED52EFCFA7F203C0A8F277
:102FD0006CC0ADF20D0EBC6F0001B6EC12F0A8C2D1
:102FE000C0F2A7C2BFF2CBEC12F00201B26B60C01C
:102FF000B3F261C0B4F20001BFDD0201C06BBF6B70
:103000000001CBEC12F00A0E0201BC6F0001B6EC1D
:1030100012F0020E0201B36FAB0EB26F00019DEC15
:1030200013F0080E0201BC6F0001B6EC12F0020EA4
:103030000201B36FAC0EB26F00019DEC13F0ABC296
:10304000AAF2ACC2A9F20201AD0706E0A751A95D40
:10305000C1E1A851AA5DBEE1AD516C5C6E02F3CF37
:10306000ADF20C0EBC6F0001B6EC12F0A8C2C0F2BB
:10307000A7C2BFF2CBEC12F00201B26B60C0B3F298
:1030800061C0B4F2000178DD0201C06BBF6B0001CA
:10309000CBEC12F00201AD2FE4D7090EBC6F00019A
:1030A000B6EC12F0020E0201B36FAB0EB26F00016C
:1030B0009DEC13F0090E0201BC6F0001B6EC12F09A
:1030C000020E0201B36FAB0EB26F00019DEC13F064
:1030D0000201A40767D7000123EF19F08CC29DF20B
:1030E0008BC29CF28AC29BF289C29AF257500408A2
:1030F0004AE102019AC292F29B51070B936F946BC3
:103100009B51F80B956F966B976B010E986F9251D0
:10311000931122E0000ED8809255906F080E9355BF
:10312000916F9F6B8FC29EF291519F5D15E303E1FA
:103130009E51905D11E29F6B90518F5D91519F590F
:10314000A16F080EA125A36FA331026E02320232D5
:103150001F0E021602509827996B9851995D12E242
:1031600097C2A1F296C2A0F295C29FF294C29EF2BB
:1031700000016ED4080E02019527000E96239723B6
:10318000992BEBD7000155EC14F09DC2B3F29CC211
:10319000B2F29BC2B1F29AC2B0F24EEC13F002014D
:1031A0009D5303E19C512F0826E29D5324E19C513D
:1031B000300821E305E19B531EE19A510D081BE302
:1031C0005750040A000105E0010A03E0030A09E080
:1031D0000FD08EC29FF28DC29EF28FC2A0F2FDD49C
:1031E00008D08EC29FF28DC29EF28FC2A0F248D547
:1031F00000D029D002015750040A000105E0010A5D
:1032000003E0030A10E01ED09DC2A1F29CC2A0F20E
:103210009BC29FF29AC29EF28EC2A3F28DC2A2F20C
:103220008FC2A4F239D69DC2A1F29CC2A0F29BC269
:103230009FF29AC29EF28EC2A3F28DC2A2F28FC2F8
:10324000A4F2A1D600D0000C62C0A1F263C0A2F229
:103250000201A36BA46B6234006E6334016EA3356C
:10326000026EA435036E0036013602360336003690
:103270000136023603360036013602360336F00ECA
:10328000001600C0A6F201C0A7F202502009A86FE4
:1032900003C0A9F203C0B2F2B16F01C0B0F200C026
:1032A000AFF20001A8EC0CF00201B26B880EB16F16
:1032B000010EB06F900EAF6F0001A8EC0CF060C073
:1032C000A0F2020161C0A1F2A26BA36B6034006E98
:1032D0006134016EA235026EA335036E00360136ED
:1032E0000236033600360136023603360036013622
:1032F00002360336F00E001600C0A5F201C0A6F299
:1033000002502009A76F03C0A8F200500609A96F58
:1033100001C0AAF2A7C2ABF203C0ACF203C0B2F282
:10332000A7C2B1F201C0B0F2AF6F0001A8EC0CF07F
:10333000000C010E0201B46F00018FEC0CF09488B8
:103340008B86030E006E002EFED78B968B86030EA7
:10335000006E002EFED78B968B86030E006E002E1D
:10336000FED78B968B86030E006E002EFED78B96B3
:103370008B86030E006E002EFED78B968B86030E77
:10338000006E002EFED78B968B86030E006E002EED
:10339000FED78B968B86030E006E002EFED78B9683
:1033A0000201A86BA8510F0814E38B86030E006E70
:1033B000002EFED782B802D0D89001D0D880A7C204
:1033C000EAFFA6C2E9FFEC52ED32ED328B96A82B54
:1033D000E9D794988B960001000CC7EC0CF08CC2D6
:1033E00063F08BC262F08AC261F089C260F02CDFA8
:1033F00002018F510208D8B0A5D1906B8F51905D1A
:10340000D8B0A0D18AC298F289C297F297533DE111
:1034100098533BE18BC29AF28CC29BF29C6B9D6BE2
:103420008B35006E8C35016E9C35026E9D35036EBA
:1034300000360136023603360036013602360336D0
:103440000036013602360336F00E001600C09FF239
:1034500001C0A0F202502009A16F03C0A2F203C074
:10346000B2F2B16F01C0B0F200C0AFF20001A8EC3F
:103470000CF00201B26B880EB16F010EB06F900EAE
:10348000AF6F0001A8EC0CF00201B26BEB0EB16F54
:10349000030EB06F800EAF6F0001A8EC0CF00201BC
:1034A000B26BBA0EB16F1B0EB06F960EAF6F00010C
:1034B000A8EC0CF00201B26BB16BB06BAF6B00010A
:1034C000A8EC0CF00201B26BB16BB06BAF6B0001FA
:1034D000A8EC0CF00201B26BBA0EB16FDB0EB06F4C
:1034E000B60EAF6F0001A8EC0CF00201B26BB16B2D
:1034F000B06BAF6B0001A8EC0CF00201B26BB16BCA
:10350000B06BAF6B0001A8EC0CF0020E0201892732
:10351000000E8A238B238C238AC298F289C297F2E9
:1035200097533DE198533BE18BC29AF28CC29BF2D8
:103530009C6B9D6B8B35006E8C35016E9C35026EDD
:103540009D35036E003601360236033600360136ED
:10355000023603360036013602360336F00E001608
:1035600000C09FF201C0A0F202502009A16F03C069
:10357000A2F203C0B2F2B16F01C0B0F200C0AFF26C
:103580000001A8EC0CF00201B26B880EB16F010EC5
:10359000B06F900EAF6F0001A8EC0CF00201B26B9F
:1035A000BA0EB16FDB0EB06FD60EAF6F0001A8EC94
:1035B0000CF00201B26BB16BB06BAF6B0001A8EC09
:1035C0000CF00201B26BB16BB06BAF6B0001A8ECF9
:1035D0000CF00201B26BBA0EB16F1B0EB06FB60EDB
:1035E000AF6F0001A8EC0CF00201B26BB16BB06BD5
:1035F000AF6B0001A8EC0CF00201B26BB16BB06BC9
:10360000AF6B0001A8EC0CF0020E02018927000E3E
:103610008A238B238C23B26B880EB16F3C0EB06F64
:10362000200EAF6F0001A8EC0CF00201B26BB16B81
:10363000B06BAF6B0001A8EC0CF0020E0201A76F9B
:10364000910EA66F000175DE0201B26B880EB16F9C
:103650003C0EB06F210EAF6F0001A8EC0CF0020120
:10366000B26BB16BB06BAF6B0001A8EC0CF0020E4B
:103670000201A76F930EA66F00015BDE0201B26B21
:10368000880EB16F3C0EB06F220EAF6F0001A8EC38
:103690000CF00201B26BB16BB06BAF6B0001A8EC28
:1036A0000CF0020E0201A76F950EA66F000141DE1D
:1036B000C7EC0CF0030E020190258F5D1EE39051C4
:1036C000902B036A8D25E96E8E510320EA6E91C21C
:1036D000EFFF9051902B036A8D25E96E8E510320E8
:1036E000EA6E9251EF6E9051902B036A8D25E96E30
:1036F0008E510320EA6E93C2EFFF030E90258F5D7B
:103700001FE39051902B036A8D25E96E8E510320A3
:10371000EA6E95C2EFFF9051902B036A8D25E96EFA
:103720008E510320EA6E9651EF6E9051902B036AF2
:103730008D25E96E8E510320EA6E9451EF6E01D013
:1037400001D05CD60001000C04008CA166D00201FF
:10375000B26BA80EB16FE70EB06F610EAF6F0001D4
:10376000A8EC0CF00201B26BB16BB06BAF6B000157
:10377000A8EC0CF00201A56BA46BA551A15D4BE375
:1037800003E1A051A45D47E204000001C7EC0CF086
:103790000201B26B800EB16F3B0EB06F010EAF6FC6
:1037A0000001A8EC0CF00201B26BB16BB06BAF6B17
:1037B0000001A8EC0CF00201B26B880EB16F3C0E58
:1037C000B06F210EAF6F0001A8EC0CF00201B26BDC
:1037D000B16BB06BAF6B0001A8EC0CF0020E0201F4
:1037E000A76FA20EA66F0001A4DD0201A42BD8B41E
:1037F000A52B000B006EA351800B036E005003102D
:1038000007E0010EB66F0001DCEC03F002D002010C
:1038100002D00201B2D789D000010201B26B200EA2
:10382000B16F050EB06F580EAF6F0001A8EC0CF031
:103830000201B26B880EB16F3B0EB06F380EAF6FE6
:103840000001A8EC0CF00201B26B200EB16F0A0E61
:10385000B06FA90EAF6F0001A8EC0CF00201B26BC3
:10386000880EB16F3B0EB06F390EAF6F0001A8EC40
:103870000CF00201B26BA80EB16FE70EB06F610ED3
:10388000AF6F0001A8EC0CF00201B26BB16BB06B32
:10389000AF6B0001A8EC0CF00201B26BB16BB06B26
:1038A000AF6B0001A8EC0CF00201B26BB16BB06B16
:1038B000AF6B0001A8EC0CF00201B26BB16BB06B06
:1038C000AF6B0001A8EC0CF0A1C2A6F20201A62B7E
:1038D000A607D8B407D0FF0EB66F0001DCEC03F0EA
:1038E0000201F6D7A0C2B6F20001DCEC03F002013F
:1038F000B26BA90EB16FE70EB06F610EAF6F000132
:10390000A8EC0CF00201B26BB16BB06BAF6B0001B5
:10391000A8EC0CF00201B26BB16BB06BAF6B0001A5
:10392000A8EC0CF0C7EC0CF002010001000C020145
:10393000B26BEB0EB16F030EB06F800EAF6F000174
:10394000A8EC0CF081DC0201936B9251935DD8B02E
:10395000B1D0976B966B69C095F268C094F26834E9
:10396000006E6934016E9635026E9735036E00362F
:10397000013602360336003601360236033600368B
:10398000013602360336F00E001600500A09996F10
:1039900001C09AF2025020099B6F03C09CF203C041
:1039A000B2F2B16F01C0B0F299C2AFF20001A8EC5F
:1039B0000CF00201B26B880EB16F3B0EB06F0A0EB5
:1039C000AF6F0001A8EC0CF0010E02019325036A11
:1039D0009025E96E91510320EA6EEFCF95F2036ACC
:1039E00093519025E96E91510320EA6EEFCF96F244
:1039F0009A6B996B95C298F296C297F29635006EC3
:103A00009535016E9935026E9A35036E0036013692
:103A100002360336003601360236033600360136EA
:103A200002360336F00E001600C09CF201C09DF273
:103A3000025020099E6F03C09FF200C0A0F201C097
:103A4000A1F2A26F03C0A3F203C0B2F2B16F01C032
:103A5000B0F200C0AFF20001A8EC0CF00201B26BB2
:103A6000B16BB06BAF6B0001A8EC0CF00201B26B54
:103A7000BB0EB16F1B0EB06F170EAF6F0001A8EC3D
:103A80000CF00201B26BB16BB06BAF6B0001A8EC34
:103A90000CF00201B26BB16BB06BAF6B0001A8EC24
:103AA0000CF07BC0A1F27AC0A0F24EDE030E020140
:103AB00093274BD700013CEF21F002019C51016A92
:103AC0009B5D03E29BC200F00CD0006A080E9D6F64
:103AD0009B3700369C51005CD8B0006E01369D2F9C
:103AE000F7D70001B5EF20F063C09FF262C09EF2ED
:103AF00061C09DF260C09CF2636A800E626E616A72
:103B0000606A24EC19F002019B6B7C509B5DD8B07D
:103B1000A3D0B26B2F0EB16FFF0EB06FF00EAF6F70
:103B20000001A8EC0CF00201B26B2F0EB16FFF0E7A
:103B3000B06FF10EAF6F0001A8EC0CF00201B26B98
:103B40002F0EB16FFF0EB06FF20EAF6F0001A8EC39
:103B50000CF00201B26BEB0EB16F030EB06F800E72
:103B6000AF6F0001A8EC0CF00201B26BB16BB06B4F
:103B7000AF6B0001A8EC0CF00201B26BBB0EB16F91
:103B80000B0EB06F370EAF6F0001A8EC0CF0020106
:103B9000B26BB16BB06BAF6B0001A8EC0CF0020123
:103BA000B26BB16BB06BAF6B0001A8EC0CF0020113
:103BB000B26BBB0EB16FDB0EB06F370EAF6F000193
:103BC000A8EC0CF00201B26BB16BB06BAF6B0001F3
:103BD000A8EC0CF00201B26BB16BB06BAF6B0001E3
:103BE000A8EC0CF00201B26BBB0EB16FEB0EB06F24
:103BF000370EAF6F0001A8EC0CF00201B26BB16B95
:103C0000B06BAF6B0001A8EC0CF00201B26BB16BB2
:103C1000B06BAF6B0001A8EC0CF00201B26BBB0EF5
:103C2000B16F1B0EB06F370EAF6F0001A8EC0CF038
:103C30000201B26BB16BB06BAF6B0001A8EC0CF082
:103C40000201B26BB16BB06BAF6B0001A8EC0CF072
:103C5000020E02019B2759D79FC263F09EC262F0F9
:103C60009DC261F09CC260F00001000C0201A36BD8
:103C7000A26B6BC0A1F26AC0A0F26A34006E6B3412
:103C8000016EA235026EA335036E00360136023690
:103C90000336003601360236033600360136023668
:103CA0000336F00E001600500A09A56F01C0A6F2F7
:103CB00002502009A76F03C0A8F203C0B2F2B16F8F
:103CC00001C0B0F2A5C2AFF20001A8EC0CF00201F5
:103CD000B26B880EB16F3B0EB06F0A0EAF6F000172
:103CE000A8EC0CF024EC19F0020E02019E6F9F6B01
:103CF0009E519D5DD8A05ED1010E9B25E96E000E00
:103D00009C21EA6EEFCFA0F29BC2E9FF9CC2EAFFC2
:103D1000EFCFA1F2A56BA46BA0C2A3F2A1C2A2F245
:103D2000A135006EA035016EA435026EA535036E77
:103D300000360136023603360036013602360336C7
:103D40000036013602360336F00E001600C0A7F228
:103D500001C0A8F202502009A96F03C0AAF200C056
:103D6000ABF201C0ACF2AD6F03C0AEF203C0B2F271
:103D7000B16F01C0B0F200C0AFF20001A8EC0CF0CE
:103D8000050E02019B25E96E000E9C21EA6EEFCF25
:103D9000A0F2020E9B25E96E000E9C21EA6EEFCF89
:103DA000A1F2A56BA46BA0C2A3F2A1C2A2F2A1359D
:103DB000006EA035016EA435026EA535036E003687
:103DC0000136023603360036013602360336003637
:103DD000013602360336F00E001600C0A7F201C00D
:103DE000A8F202502009A96F03C0AAF200500109ED
:103DF000AB6F01C0ACF2A9C2ADF203C0AEF203C01A
:103E0000B2F2A9C2B1F201C0B0F2AF6F0001A8ECEA
:103E10000CF0040E02019B25E96E000E9C21EA6E57
:103E2000EFCFA0F2030E9B25E96E000E9C21EA6EF7
:103E3000EFCFA1F2A56BA46BA0C2A3F2A1C2A2F224
:103E4000A135006EA035016EA435026EA535036E56
:103E500000360136023603360036013602360336A6
:103E60000036013602360336F00E001600C0A7F207
:103E700001C0A8F202502009A96F03C0AAF20050A5
:103E80000209AB6F01C0ACF2A9C2ADF203C0AEF241
:103E900003C0B2F2A9C2B1F201C0B0F2AF6F00012B
:103EA000A8EC0CF00201B26BEB0EB16F030EB06F19
:103EB000800EAF6F0001A8EC0CF00201B26BB16B89
:103EC000B06BAF6B0001A8EC0CF00201B26BBB0E43
:103ED000B16F0B0EB06F370EAF6F0001A8EC0CF096
:103EE0000201B26BB16BB06BAF6B0001A8EC0CF0D0
:103EF0000201B26BB16BB06BAF6B0001A8EC0CF0C0
:103F00000201B26BBB0EB16FDB0EB06F370EAF6F3D
:103F10000001A8EC0CF00201B26BB16BB06BAF6B9F
:103F20000001A8EC0CF00201B26BB16BB06BAF6B8F
:103F30000001A8EC0CF00201B26BBB0EB16FEB0EEE
:103F4000B06F370EAF6F0001A8EC0CF00201B26B3E
:103F5000B16BB06BAF6B0001A8EC0CF00201B26B5F
:103F6000B16BB06BAF6B0001A8EC0CF00201B26B4F
:103F7000BB0EB16F1B0EB06F370EAF6F0001A8EC18
:103F80000CF00201B26BB16BB06BAF6B0001A8EC2F
:103F90000CF00201B26BB16BB06BAF6B0001A8EC1F
:103FA0000CF0020E02019E27060E9F279B27000E93
:103FB0009C239ED69DA1CAD0010E9B25E96E000EC2
:103FC0009C21EA6EEFCFA0F29BC2E9FF9CC2EAFF00
:103FD000EFCFA1F2A56BA46BA0C2A3F2A1C2A2F283
:103FE000A135006EA035016EA435026EA535036EB5
:103FF0000036013602360336003601360236033605
:104000000036013602360336F00E001600C0A7F265
:1040100001C0A8F202502009A96F03C0AAF200C093
:10402000ABF201C0ACF2AD6F03C0AEF203C0B2F2AE
:10403000B16F01C0B0F200C0AFF20001A8EC0CF00B
:10404000020E02019B25E96E000E9C21EA6EEFCF65
:10405000A0F2A26BA0C2A1F2A035026EA235036E3F
:10406000023603360236033602360336F00E0216E7
:1040700002C0A4F203C0A5F2200EA66FA76B0250E7
:104080000109A86F03C0A9F2A6C2AAF2A7C2ABF2A7
:10409000A7C2B2F2A6C2B1F203C0B0F2AF6F000184
:1040A000A8EC0CF00201B26BEB0EB16F030EB06F17
:1040B000800EAF6F0001A8EC0CF00201B26BB16B87
:1040C000B06BAF6B0001A8EC0CF00201B26BBB0E41
:1040D000B16F0B0EB06F370EAF6F0001A8EC0CF094
:1040E0000201B26BB16BB06BAF6B0001A8EC0CF0CE
:1040F0000201B26BB16BB06BAF6B0001A8EC0CF0BE
:104100000201B26BBB0EB16FDB0EB06F370EAF6F3B
:104110000001A8EC0CF00201B26BB16BB06BAF6B9D
:104120000001A8EC0CF00201B26BB16BB06BAF6B8D
:104130000001A8EC0CF00201B26BE80EB16F030EA7
:10414000B06F060EAF6F0001A8EC0CF079C0A1F2C1
:1041500078C0A0F20001A4EC1BF0000C96C29BF208
:10416000030E02019C6F0001A8D401C09AF2D890FE
:104170007D34020190159B6F9C6B9D6B9E6BD8905C
:104180009E319D319C319B31986F985325E0985119
:104190007C5C996F00018CA301D0A6DC02019951CF
:1041A0009A5D02E29AC299F295C29CF294C29BF285
:1041B00099C29DF200015ADD020199519A5F99510D
:1041C000030DF3509427000E9523D890993560265F
:1041D000000E6122622263227C509A5D19E395C22F
:1041E0009CF294C29BF27CC09DF200013FDD7C50AA
:1041F000030DF35002019427000E95237C509A5F23
:10420000D8907C346026000E612262226322E4D7BB
:104210009A530CE000018CA301D066DC95C29CF29D
:1042200094C29BF29AC29DF221DD020100014DEF82
:1042300021F0C7EC0CF08CC263F08BC262F08AC232
:1042400061F089C260F08BC291F28CC292F20201DD
:10425000936B946B8B51F80810E192530EE19353DA
:104260000CE194530AE18EC291F28DC290F28FC29A
:1042700092F2000197EF1CF010D08CC293F28BC227
:1042800092F28AC291F289C290F28EC295F28DC2E8
:1042900094F28FC296F2000161D7000C6AC0A7F2B7
:1042A0004CEC07F062C0B6F2DCEC03F063C0BDF288
:1042B00006EC05F06B5204E06BC0A7F24CEC07F083
:1042C00069C0BDF206EC05F0000CE8DF010E6024C9
:1042D00002019C6F000E61209D6FA36F9CC2A2F231
:1042E000000132EC10F0000C8AC294F289C293F201
:1042F0008EC292F28DC291F294C2A3F293C2A2F244
:1043000032EC10F0D89002018F33906B8F51905D9A
:104310001AE2D8909035036A9125E96E92510320F4
:10432000EA6EECCF96F2ED52EFCF95F2020EA46F4B
:1043300096C2A6F295C2A5F2000128EC10F0C5DFE6
:104340000201902BE3D70001000C02019651070BEC
:104350009C6F4F5012082EE1F80E96173F0E9717DC
:104360009B6B9C519B5D26E297C203F09651962B66
:10437000D8B4972BA06F03C0A1F203C0A3F2A26F21
:10438000000132EC10F0040E0201A06F020EA26FC9
:104390009D0EA16F00017EEC12F0020E0201A46FCF
:1043A0009EC2A6F29DC2A5F2000128EC10F0020107
:1043B0009B2BD7D79B6B9A519B5D2DE297C203F045
:1043C0009651962BD8B4972BA06F03C0A1F203C0CF
:1043D000A3F2A26F000132EC10F0020199C203F0C7
:1043E00098C200F0020E9827D8B0992B00C0E9FFC0
:1043F00003C0EAFFECCFA1F2ED52EFCFA0F2020E24
:10440000A46FA1C2A6F2A0C2A5F2000128EC10F090
:1044100002019B2BD0D74F50120837E17450975DA3
:1044200007E303E17350965D03E3040E9F6F02D030
:10443000080E9F6F9C519A279F519A5D26E297C262
:1044400003F09651962BD8B4972BA06F03C0A1F21E
:1044500003C0A3F2A26F000132EC10F0040E0201BF
:10446000A06F020EA26F9D0EA16F00017EEC12F0F4
:10447000020E0201A46F9EC2A6F29DC2A5F2000127
:1044800028EC10F002019A2BD7D70001000C8AC249
:1044900093F289C292F28EC295F28DC294F2D890B4
:1044A00002018F339251070B006E0050FF0A090F73
:1044B000916F91518F5D02E28FC291F293511F086B
:1044C00043E2FF0A03E1925103083EE2906B8F51F1
:1044D000905D39E293C203F09251922BD8B4932BA2
:1044E000966F03C097F203C0A3F2A26F000132ECF3
:1044F00010F0020195C203F094C200F0020E94275E
:10450000D8B0952B00C0E9FF03C0EAFFECCF97F2CB
:10451000ED52EFCF96F2020EA46F97C2A6F296C2AA
:10452000A5F2000128EC10F0080E0201A76F0001AF
:104530004CEC07F0060E0201B66F0001DCEC03F054
:104540000201902BC4D741D093C297F292C296F247
:104550008EC299F28DC298F291C29AF20001F5DEF4
:10456000B4DE020191518F5FD89091359427000EEF
:104570009523080E906F90518F5D15E361C097F2FF
:1045800060C096F295C299F294C298F2080E9A6FA2
:104590000001DBDE9ADE100E02019427000E952347
:1045A000080E9027E8D7070E8F178F530EE061C0D3
:1045B00097F260C096F295C299F294C298F28FC2B7
:1045C0009AF20001C2DE81DE02010001000C02014C
:1045D0009B6B010E9A5D9B5D2AE299C203F098C223
:1045E00000F0020E9827D8B0992B00C0E9FF03C055
:1045F000EAFFECCF9DF2ED52EFCF9CF2020EA46FDA
:104600009DC2A6F29CC2A5F2000128EC10F0010E9A
:10461000602402019C6F000E61209D6FA36F9CC2FD
:10462000A2F2000132EC10F002019B2BD2D799C20A
:1046300003F098C2E9FF99C2EAFFECCF9DF2ED5278
:10464000EFCF9CF2020EA46F9DC2A6F29CC2A5F20F
:10465000000128EC10F039DE000C8AC297F289C202
:1046600096F28EC293F28DC292F2D89002018F33ED
:104670007450975D09E303E17350965D05E37DC0D7
:1046800094F27EC095F204D07BC094F27CC095F287
:1046900096519515916F97C2A3F296C2A2F20001AE
:1046A00032EC10F00201915318E09151945D906F3B
:1046B00090518F5D02E28FC290F293C299F292C242
:1046C00098F290C29AF2000182DF020190518F5F4E
:1046D000D89090359227000E932394518F5D11E36B
:1046E00093C299F292C298F294C29AF200016FDFDB
:1046F000D890020194359227000E932394518F5F36
:10470000ECD78F5309E093C299F292C298F28FC20C
:104710009AF200015CDF02010001000C8AC298F2EB
:1047200089C297F28EC291F28DC290F2D8900201A6
:104730008F338F53D8B46ED098C203F09751972B14
:10474000D8B4982B996F03C09AF203C0A3F2A26F5A
:10475000000132EC10F0020191C203F090C200F0AF
:10476000020E9027D8B0912B00C0E9FF03C0EAFFEA
:10477000ECCF03F0ED52EFCF92F203C093F29851D9
:104780001F0808E2FF0A03E19751070803E281C00E
:1047900096F22ED080C096F2020EA46F93C2A6F2BB
:1047A00092C2A5F2000128EC10F078DD040E02019F
:1047B000A06F020EA26F940EA16F00017EEC12F0AA
:1047C0000201960706E09251945DE6E19351955DF2
:1047D000E3E19251945D0BE19351955D08E19651AF
:1047E0000001805D8203F3CF96F2020101D012D066
:1047F00096519607000A0CE0020EA46F93C2A6F22F
:1048000092C2A5F2000128EC10F048DD0201F0D7B9
:104810008F078FD70001000C000CEA6A280EE96EA2
:1048200085C28CF284C28BF283C28AF282C289F280
:1048300087C28EF286C28DF288C28FF235EC02F00A
:104840008B968B98000C02018C6B8B6B200E8A6F01
:10485000070E896F020E8E6F800E8D6F020E8F6FA6
:1048600000018AEC12F0FDEC10F0FF0E0201801343
:104870000F0E8113856B846B200E836F070E826F82
:10488000020E876F800E866F020E886F0001C5DFF3
:10489000000CD9DF03EC11F0000C7EC2A7F24CEC47
:1048A00007F0080E0201886F80C289F20001B6ECA1
:1048B00010F002017F5306E07FC2A7F200014CEC2A
:1048C00007F002010001000C6CC07EF26DC07FF2A7
:1048D00066C080F2E2DF000C6EC07EF26FC07FF235
:1048E00067C080F2DADF000C016A026A006A036ABC
:1048F00002018B5102E18A5118E0100E8C6FD890A2
:1049000088378937003603368B51035C02E18A51C0
:10491000005C07E38A51005ED8A003068B51035E5A
:10492000D880013602368C2FEAD70001A2EF24F09E
:1049300082C289F281C288F202018B6B83C28AF241
:104940000001D2D702C087F201C086F20201856B56
:10495000846B8551875D26E303E18651845D22E205
:1049600004007EC288F280C289F20001B6EC10F029
:1049700002017F5306E07FC2A7F200014CEC07F072
:10498000020183516024886F000E6120896FA36F3C
:1049900088C2A2F2000132EC10F00201842BD8B4DC
:1049A000852BD7D70001000C6CC07EF26DC07FF262
:1049B00066C080F2200E0201826F816B7FC083F29D
:1049C0000001B6DF000C6EC07EF26FC07FF267C0E0
:1049D00080F2010E0201826F816B836F0001A8DFFC
:1049E000000C6CC07EF26DC07FF266C080F20201E6
:1049F000826B7FC081F27FC083F2000199DF78C0B3
:104A0000A3F277C0A2F232EC10F0020E0201A46F02
:104A10003F0EA66FFF0EA56F000128EC10F0C4DF5B
:104A20000201A36BA26B000132EC10F0030E020135
:104A3000A46FA66BFF0EA56F000128EC10F0C3DF7A
:104A4000000C25EC11F078C0A3F277C0A2F232EC92
:104A500010F0FDEC10F003EC11F0000C0201B96B4A
:104A60003C0EB86FB76B040EB66F0001E3EC12F0AA
:104A70000C0E0201BC6F0001B6EC12F085C2C0F250
:104A800084C2BFF2CBEC12F00201BC6B0001B6ECA9
:104A900012F00201C06BBF6B0001CBEC12F00201FF
:104AA000BC6B0001B6EC12F0645066240201866F04
:104AB000B66F0001DCEC03F0655067240201866FDD
:104AC00086C2BDF2000106EC05F00201C06BBF6BAF
:104AD0000001CBEC12F0000C0201856B830E846F99
:104AE0000001BCDF880E02017E6F7E518F0808E353
:104AF000856B7EC284F20001B1DF02017E2BF5D707
:104B00000001000C0201856B810E846F0001A6DF9D
:104B1000000C0201856B800E846F00019FDF000C8A
:104B2000EA6A2A0EE96E85C28CF284C28BF283C2D5
:104B30008AF282C289F287C28EF286C28DF288C260
:104B40008FF235EC02F08B968B98000C0201B96B5A
:104B50003C0EB86FB76B050EB66F0001E3EC12F0B8
:104B60000C0E0201BC6F0001B6EC12F083C2C0F261
:104B700082C2BFF2CBEC12F083C285F282C284F211
:104B80006DDF000C0201856B200E846F836B826BDE
:104B9000020E876F800E866F020E886F0001C0DFE5
:104BA0007FC283F27EC282F2D1DF000C02017F6BF2
:104BB000810E7E6F0001E6DF02017F6B820E7E6F49
:104BC0000001E0DF010E0201836F800E826F0001A1
:104BD000BDDF020E0201836F800E826F0001B6DF1F
:104BE000040E0201836F800E826F0001AFDF080E9A
:104BF0000201836F800E826F0001A8DF100E020198
:104C0000836F800E826F0001A1DF200E0201836F8F
:104C1000800E826F00019ADF400E0201836F800ECA
:104C2000826F000193DF800E0201836F826F0001AB
:104C30008DDF000CFF0E02017F6F870E7E6F00017B
:104C4000A1DF55EC14F00201B36B200EB26FB16B13
:104C5000B06B00014EEC13F09FEC14F0000C02015D
:104C6000836B840E826F000171DF000C010E020164
:104C7000836F8A0E826F000169DF000CF7DF000C82
:104C8000010E0201836F800E826F00015FDF020E52
:104C90000201806FC80EB66F0001DCEC03F0020168
:104CA000802FF8D70001000C0201836B820E826F07
:104CB00000014CDF0201856B200E846F836B280E90
:104CC000826F020E876F7E0E866F020E886F000164
:104CD00027DF340E0201806F000125EC0FF0D0DFDA
:104CE000000C80C28DF281C28EF202018F6B906B3C
:104CF0008035006E8135016E8F35026E9035036E02
:104D000000360136023603360036013602360336E7
:104D10000036013602360336F00E00160050060942
:104D2000926F01C093F202502009946F03C095F274
:104D300003C0B2F2B16F01C0B0F292C2AFF2000193
:104D4000A8EC0CF00201B26B880EB16F3B0EB06F95
:104D5000260EAF6F0001A8EC0CF002017EC28CF2AF
:104D60007FC28DF28E6B8F6B7E35006E7F35016E4C
:104D70008E35026E8F35036E0036013602360336ED
:104D80000036013602360336003601360236033667
:104D9000F00E001600500609916F01C092F2025009
:104DA0002009936F03C094F203C0B2F2B16F01C047
:104DB000B0F291C2AFF20001A8EC0CF00201B26BAC
:104DC000880EB16F3B0EB06F160EAF6F0001A8ECEE
:104DD0000CF002018635026E8735036E023603360B
:104DE0000236033602360336F00E02160250070969
:104DF0008D6F03C08EF2200E906B90C2B2F2B16F35
:104E000003C0B0F28DC2AFF20001A8EC0CF00201B9
:104E10008B6B8A6B8B51895D6FE303E188518A5DEF
:104E20006BE28235006E8335016E8435026E853506
:104E3000036E00360136023603360036013602367E
:104E400003360036013602360336F00E00160050E7
:104E50000A098D6F01C08EF2025020098F6F03C0C6
:104E600090F203C0B2F2B16F01C0B0F28DC2AFF2E6
:104E70000001A8EC0CF00201B26B880EB16F3B0E82
:104E8000B06F0A0EAF6F0001A8EC0CF077C0A1F272
:104E900076C0A0F2A4EC1BF00201B26B430EB16F1E
:104EA000030EB06F070EAF6F0001A8EC0CF002010B
:104EB000B26BAF0EB16FB06B420EAF6F0001A8ECDA
:104EC0000CF00201B26BEC0EB16F270EB06F640EE6
:104ED000AF6F0001A8EC0CF00201B26B880EB16F4D
:104EE0003B0EB06F160EAF6F0001A8EC0CF0020184
:104EF0008A2BD8B48B2B8ED70001000C0201816B5A
:104F0000806B7F6B7E6B856B846B6FC083F26EC032
:104F100082F2876B7EC086F280C089F27FC088F201
:104F20000001DFDE8CA302D074EC1DF00201816B66
:104F3000800E806F7F6B7E6B856B846B6FC083F29E
:104F40006EC082F2876B7EC086F282C089F281C019
:104F500088F20001C6DE000C8CA302D074EC1DF0B8
:104F60000201816B806B73C07FF272C07EF272347B
:104F7000006E7334016E8035026E8135036E00362B
:104F80000136023603360036013602360336003665
:104F9000013602360336F00E001600500A09836F00
:104FA00001C084F202502009856F03C086F203C05D
:104FB000B2F2B16F01C0B0F283C2AFF20001A8EC4F
:104FC0000CF00201B26B880EB16F3B0EB06F0A0E8F
:104FD000AF6F0001A8EC0CF075C0A1F274C0A0F294
:104FE000A4EC1BF0000CB8DF895302E18A5302E005
:104FF0008B5301E10FD002018C6BF80E8B6F8A6B23
:10500000896B8AC08EF289C08DF28BC08FF200014D
:1050100019EC21F0000C0201B26B200EB16F080EEA
:10502000B06F060EAF6F0001A8EC0CF00201B26B7E
:10503000880EB16F3B0EB06F260EAF6F0001A8EC6B
:105040000CF00201B26B200EB16FB06B060EAF6FA9
:105050000001A8EC0CF00201B26B880EB16F3B0EA0
:10506000B06F160EAF6F0001A8EC0CF0BCDF000CA7
:105070000201816B7F0E806FF00E7F6F7E6B856B00
:10508000846B71C083F270C082F286C087F285C0E3
:1050900086F288C089F287C088F2000122DE000C07
:1050A0002DDF0201B26B240EB16F040EB06FDA0E69
:1050B000AF6F0001A8EC0CF00201B26B880EB16F6B
:1050C0003B0EB06F0A0EAF6F0001A8EC0CF075C07C
:1050D000A1F274C0A0F2A4EC1BF00201B26B240E8A
:1050E000B16F040EB06FCA0EAF6F0001A8EC0CF0E8
:1050F0000201B26B880EB16F3B0EB06F0A0EAF6F3C
:105100000001A8EC0CF075C0A1F274C0A0F2A4ECF0
:105110001BF0000C000C02017D51000105E0010AAA
:105120000EE0030A17E021D0EA6A300EE96E35EC92
:1051300002F0EA6A360EE96E35EC02F016D0EA6A41
:10514000320EE96E35EC02F0EA6A380EE96E35ECA3
:1051500002F00BD0EA6A340EE96E35EC02F0EA6A2E
:105160003A0EE96E35EC02F000D08B968B98BCEFCE
:1051700028F081C17DF2CFD7070E0101806F010EAB
:105180000A6E000191EC02F0B5EF2EF00201806B87
:1051900083C17FF282C17EF281C17DF2040E0A5C7E
:1051A000816F80C285F27FC284F27EC283F27DC2AB
:1051B00082F2010E876F840E866F81C288F2000131
:1051C0000DEC24F0070E0101806F010E0A6E000144
:1051D00091EC02F0B5EF2EF00201806B83C17FF2FB
:1051E00082C17EF281C17DF20A50060803E184C1CA
:1051F0000AF002D084C10AF080C285F27FC284F234
:105200007EC283F27DC282F2010E876F840E866FAA
:105210000AC088F2000184DCC40E0101806F040E14
:105220000A26000191EC02F0B5EF2EF086C28EF254
:1052300085C28DF202018A6B89518A5D26E28EC297
:1052400003F08D518D2BD8B48E2B8F6F03C090F24D
:1052500003C0A3F2A26F000132EC10F0050E0201B0
:10526000A06F020EA26F8B0EA16F00017EEC12F0F8
:1052700002018A518725016E000E882101C0E9FFD5
:10528000EA6E8BC2EFFF8A2BD7D70001000C6AC0F1
:10529000A7F24CEC07F064C0B6F2DCEC03F065C09A
:1052A000BDF206EC05F06B5204E06BC0A7F24CECCB
:1052B00007F0010E602402018D6F000E61208E6FD9
:1052C000A36F8DC2A2F2000132EC10F08BEF29F037
:1052D00086C28CF285C28BF28CC2A3F28BC2A2F280
:1052E00032EC10F002018A6B89518A5D17E28A5113
:1052F0008725016E000E8821036E01C0E9FFEA6E6A
:10530000EFCF8DF2030EA46FA66B8DC2A5F2000144
:1053100028EC10F0BCD702018A2BE6D70001000C64
:10532000C7EC0CF0020185C260F086C261F07F0E0E
:10533000626E636A000124EC19F00201B26BEB0E9D
:10534000B16F030EB06F800EAF6F0001A8EC0CF0D0
:1053500002018951010842E28A6B89518A5D3EE26D
:10536000B26BBA0EB16F0B0EB06FB60EAF6F00011D
:10537000A8EC0CF00201B26BB16BB06BAF6B00012B
:10538000A8EC0CF00201B26BB16BB06BAF6B00011B
:10539000A8EC0CF00201B26B880EB16F3C0EB06F3E
:1053A000200EAF6F0001A8EC0CF00201B26BB16BE4
:1053B000B06BAF6B0001A8EC0CF002018A5187259D
:1053C0008B6F000E88218C6FA76F8BC2A6F2000135
:1053D00099EC19F0020E02018A27BFD70001000CD8
:1053E0000201956B946B6DC093F26CC092F26C34B9
:1053F000006E6D34016E9435026E9535036E003685
:1054000001360236033600360136023603360036E0
:10541000013602360336F00E001600500A09976F67
:1054200001C098F202502009996F03C09AF203C09C
:10543000B2F2B16F01C0B0F297C2AFF20001A8ECB6
:105440000CF00201B26B880EB16F3B0EB06F0A0E0A
:10545000AF6F0001A8EC0CF024EC19F00201B26B64
:10546000EB0EB16F030EB06F800EAF6F0001A8ECB2
:105470000CF00201916BD89090379051915D59E2F8
:10548000010E9125036A8E25E96E8F510320EA6E85
:10549000EFCF93F2036A91518E25E96E8F5103206D
:1054A000EA6EEFCF94F2986B976B93C296F294C228
:1054B00095F29435006E9335016E9735026E9835EE
:1054C000036E0036013602360336003601360236E8
:1054D00003360036013602360336F00E001600C0E1
:1054E0009AF201C09BF2025020099C6F03C09DF20A
:1054F00003C0B2F2B16F01C0B0F200C0AFF2000160
:10550000A8EC0CF00201B26BB16BB06BAF6B000199
:10551000A8EC0CF00201B26BBB0EB16F1B0EB06FAA
:10552000170EAF6F0001A8EC0CF0020E02019127DC
:10553000A4D779C0A1F278C0A0F20001A4EC1BF0BE
:10554000000CC7EC0CF0020185C260F086C261F06D
:105550007F0E626E636AD8908933D89000018435DB
:10556000020185158D6F8E6BD8908E318D318B6FCA
:105570008B5321E08B510001835D02018C6F8C51B4
:10558000895D02E289C28CF288C28FF287C28EF2F4
:105590008CC290F2000124DF02018C51895FD89007
:1055A0008C358727000E8823D8908C356026000E16
:1055B00061226222632283C08AF28A51895D1CE3E0
:1055C00088C28FF287C28EF283C090F2000108DF9A
:1055D000D890833502018727000E8823000183516C
:1055E00002018A27D890000183356026000E6122CF
:1055F000622263220201E1D78951000184150DE086
:10560000020189510001841502018D6F88C28FF259
:1056100087C28EF2906F0001E3DE000C0201BC6BCA
:105620000001B6EC12F0800E0201C06FA60EBF6F33
:105630000001CBEC12F00201BC6B0001B6EC12F0E1
:10564000500E0201C06FA80EBF6F0001CBEC12F02C
:105650000201BC6B0001B6EC12F06E0E0201C06FCD
:10566000F50EBF6F0001CBEC12F00201BC6B000124
:10567000B6EC12F00201C06BBF6B0001CBEC12F074
:10568000020E0201BC6F0001B6EC12F090C2B3F240
:105690008FC2B2F29DEC13F0000C86C28CF285C270
:1056A0008BF20201BC6B0001B6EC12F09E0E0201FF
:1056B000C06FA60EBF6F0001CBEC12F00201BC6BF5
:1056C0000001B6EC12F09C0E0201C06FA60EBF6F77
:1056D0000001CBEC12F002018A6B89518A5D59E21C
:1056E000BC6B0001B6EC12F002018BC200F0036A41
:1056F0008BC28DF203500E098E6FC06F8BC2BFF24A
:105700000001CBEC12F00201BC6B0001B6EC12F010
:105710006E0E0201C06FA90EBF6F0001CBEC12F03C
:105720000201BC6B0001B6EC12F08CC28DF20201DA
:105730008E6B8CC200F0036A8CC28FF203500E098C
:10574000906FC06F8CC2BFF20001CBEC12F002016F
:105750008B2BD8B48C2BBC6B0001B6EC12F06E0E08
:105760000201C06FAA0EBF6F0001CBEC12F0020164
:1057700088C203F08751872BD8B4882B8D6F03C064
:105780008EF203C090F28F6F000148DF02018A2B76
:10579000A4D70001000C0201BC6B0001B6EC12F0B2
:1057A00002018FC290F20E0EC06F8FC2BFF20001D5
:1057B000CBEC12F00201BC6B0001B6EC12F06E0EE5
:1057C0000201C06FA80EBF6F0001CBEC12F0020106
:1057D000BC6B0001B6EC12F0840E0201C06FA60E85
:1057E000BF6F0001CBEC12F00201BC6B0001B6EC04
:1057F00012F00E0E0201C06F550EBF6F0001CBEC10
:1058000012F00201BC6B0001B6EC12F06E0E020148
:10581000C06FA70EBF6F0001CBEC12F00201BC6B92
:105820000001B6EC12F00E0E0201C06FAA0EBF6F9F
:105830000001CBEC12F00201BC6B0001B6EC12F0DF
:105840006E0E0201C06FA70EBF6F0001CBEC12F00D
:105850000201BC6B0001B6EC12F0820E0201C06FB7
:10586000A60EBF6F0001CBEC12F06FA221D0020197
:10587000BC6B0001B6EC12F00201C06BBF6B000103
:10588000CBEC12F00201BC6B0001B6EC12F002018D
:10589000C06BBF6B0001CBEC12F069EC14F064C07C
:1058A000B6F2DCEC03F065C0BDF206EC05F027D0E3
:1058B0000201BC6B0001B6EC12F00201C06BBF6BC1
:1058C0000001CBEC12F00201BC6B0001B6EC12F04F
:1058D000645066240201906FB66F0001DCEC03F0A7
:1058E000655067240201906F90C2BDF2000106EC82
:1058F00005F00201C06BBF6B0001CBEC12F002019E
:10590000BC6B0001B6EC12F0940E0201C06FA60E43
:10591000BF6F0001CBEC12F0000C86C28DF285C285
:105920008CF20201BC6B0001B6EC12F09E0E02017B
:10593000C06FA60EBF6F0001CBEC12F00201BC6B72
:105940000001B6EC12F09C0E0201C06FA60EBF6FF4
:105950000001CBEC12F002018A6B89518A5D58E29A
:10596000BC6B0001B6EC12F002018CC200F0036ABD
:105970008CC28EF203500E098F6FC06F8CC2BFF2C3
:105980000001CBEC12F00201BC6B0001B6EC12F08E
:105990006E0E0201C06FA90EBF6F0001CBEC12F0BA
:1059A0000201BC6B0001B6EC12F08DC28EF2020156
:1059B0008F6B8DC200F0036A8DC290F203500E0906
:1059C000916FC06F8DC2BFF20001CBEC12F00201EB
:1059D0008C2BD8B48D2BBC6B0001B6EC12F06E0E84
:1059E0000201C06FAA0EBF6F0001CBEC12F0036A78
:1059F00002018A518725E96E88510320EA6EEFCFB4
:105A00008EF28EC28FF20001C6DE02018A2BA5D76C
:105A10000001000C86C28CF285C28BF20201BC6BC5
:105A20000001B6EC12F09E0E0201C06FA60EBF6F11
:105A30000001CBEC12F00201BC6B0001B6EC12F0DD
:105A40009C0E0201C06FA60EBF6F0001CBEC12F0DE
:105A500002018A6B89518A5D39E2BC6B0001B6ECA8
:105A600012F002018CC203F08B518B2BD8B48C2B1B
:105A70008D6F03C08EF2006E036A8F6F03500E09A4
:105A8000906FC06F8DC2BFF20001CBEC12F002012B
:105A9000BC6B0001B6EC12F06E0E0201C06FA90ED5
:105AA000BF6F0001CBEC12F0020188C203F08751F6
:105AB000872BD8B4882B8D6F03C08EF203C090F271
:105AC0008F6F0001ABDD02018A2BC4D70001000CEF
:105AD00086C28CF285C28BF20201BC6B0001B6EC6F
:105AE00012F09E0E0201C06FA60EBF6F0001CBEC3C
:105AF00012F00201BC6B0001B6EC12F09C0E020128
:105B0000C06FA60EBF6F0001CBEC12F002018A6BD2
:105B100089518A5D38E2BC6B0001B6EC12F00201DB
:105B20008CC203F08B518B2BD8B48C2B8D6F03C0A0
:105B30008EF2006E036A8F6F03500E09906FC06F74
:105B40008DC2BFF20001CBEC12F00201BC6B000170
:105B5000B6EC12F06E0E0201C06FA90EBF6F00010D
:105B6000CBEC12F0036A02018A518725E96E885155
:105B70000320EA6EEFCF8DF28DC28FF200010BDEB3
:105B800002018A2BC5D70001000C000CEA6A2C0E1A
:105B9000E96E81C286F280C285F283C288F282C237
:105BA00087F284C289F235EC02F08B968B98EDEF88
:105BB0002DF082C17EF281C17DF2030E0A5C0201EA
:105BC0007F6F7EC281F27DC280F2010E836F830EF1
:105BD000826F7FC284F20001D9D7070E0101806F66
:105BE000010E0A6E000191EC02F0B5EF2EF0EA6AA8
:105BF0002E0EE96E80C286F27FC285F282C288F2E2
:105C000081C287F283C289F235EC02F08B968B98C1
:105C10001DEF2EF082C17EF281C17DF283C10AF0B8
:105C20007EC280F27DC27FF2010E0201826F830E7E
:105C3000816F0AC083F20001DAD7E20E0101806FA2
:105C4000030E0A26000191EC02F0B5EF2EF0BAEC3B
:105C500003F0D00E0101806F816B826B836B846BCC
:105C6000050E0A6E000191EC02F0B5EF2EF0E7ECA4
:105C700006F0D00E0101806F010E816F826B836B85
:105C8000846B050E0A6E000191EC02F0B5EF2EF068
:105C9000010E02017C6F7B5301E06AD0010180514B
:105CA000110803E100016FEF04F08051120803E1D5
:105CB0000001B2EF04F08051140803E1000151EF3C
:105CC00005F08051150805E1000118EC05F04DD0F4
:105CD000010180511A0803E1000165EF05F08051D0
:105CE0001B0803E1000170EF05F080511C0803E17F
:105CF0000001DAEF05F08051410803E1000165EF92
:105D00000FF08051B20803E1000188EF0FF08051DD
:105D1000470803E10001A9EF0FF08051430803E1B8
:105D20000001B9EF28F08051420803E10001C6EFFD
:105D300028F08051440803E10001ECEF28F0805185
:105D4000450802E1000135D78051460802E1000113
:105D500061D78051500802E1000179D78051510884
:105D600002E1000184D702017C6B02017CC201F0D8
:105D70000001C7EF3FF00201BC8104009488850E4A
:105D8000006E002EFED782A80FD00400BB51BB07C7
:105D9000000A03E1BC9108D006D0FF0EBD6F0001E0
:105DA00006EC05F00201EFD7000EBCB1010E016E4A
:105DB0000001000C100E0201A96F9488FF0EBB6F4A
:105DC0000001D9DF0201AB6BAA6BAB510001905D02
:105DD0000CE305E10201AA5100018F5D06E3020117
:105DE000AA2BD8B4AB2BF1D700018B860201AD6B87
:105DF000AC6BAD510001905D10E305E10201AC51C7
:105E000000018F5D0AE3030E006E002EFED7020133
:105E1000AC2BD8B4AD2BEDD7000182B802D0D8900E
:105E200001D0D8800201A737A8379498D890A53719
:105E3000A63702E28B9801D08B888B96AF6BAE6B46
:105E4000AF510001905D11E305E10201AE51000187
:105E50008F5D0BE3110E006E002EFED700D0020105
:105E6000AE2BD8B4AF2BECD7000194880201A90760
:105E7000D8B402D00001B9D7A7C201F0A8C202F07D
:105E80000001000C050E906F940E8F6FFF0E020143
:105E9000BB6F000170DF015268E0100E0201A66FB7
:105EA000A56B000187DF948882B8FED78B86926B42
:105EB000010E916F82B808D0912BD8B4922B9151DA
:105EC000921102E00400F6D782B808D0912BD8B422
:105ED000922B9151921102E00400F6D70201A46BBB
:105EE000A36BA26BA16B82A80ED0A12BD8B0A22B62
:105EF000D8B0A32BA151A211A31105E01E0E006E74
:105F0000002EFED7F0D78B96915192112AE0020114
:105F1000A15309E1A25307E1A35305E1A453D8A477
:105F200002D000011ED0A431036EA331026EA23153
:105F3000016EA131006E03320232013200320332AF
:105F400002320132003203320232013200320332B5
:105F500002320132003200C08FF0000101C090F027
:105F600004D0050E906F940E8F6F0201A1C201F054
:105F7000A2C202F00001000CFF0E0201BB6F000183
:105F8000FADE02019BC200F09C510F0B036E9BC214
:105F9000A1F203505009A26FA66F9BC2A5F20001A7
:105FA00009DF0201A06B9F51A05D1FE2FF0EBB6FD6
:105FB0000001E1DE015213E09EC203F002019DC226
:105FC000E9FF9EC2EAFFEFCFA1F2600EA66FA1C269
:105FD000A5F20001EFDE93A301D054DF00D002014F
:105FE0009D2BD8B49E2BA02BDED70001000C020104
:105FF0009A6B9AC299F29851745C09E303E1735069
:10600000975D05E298518009996F97C29AF286C010
:106010009CF285C09BF2020E9E6F990E9D6F010E41
:106020009F6F0001A9DF88C09CF287C09BF2020E1F
:1060300002019E6F9A0E9D6F010E9F6F00019CDF03
:10604000000C080E0201946F9488FF0EBB6F0001D4
:1060500092DE0201966B956B96510001905D0CE308
:1060600005E10201955100018F5D06E30201952BC8
:10607000D8B4962BF1D700018B860201986B976BF1
:1060800098510001905D10E305E102019751000174
:106090008F5D0AE3030E006E002EFED70201972BE0
:1060A000D8B4982BEDD7000182B802D0D89001D097
:1060B000D880020193379498D890923702E28B9857
:1060C00001D08B888B969A6B996B9A510001905DE9
:1060D00011E305E10201995100018F5D0BE3110EFF
:1060E000006E002EFED700D00201992BD8B49A2B57
:1060F000ECD70001948802019407D8B402D00001C3
:10610000BBD793C201F00001000C0201916BFF0E9E
:10611000BB6F000130DE015206E00201926B00010C
:1061200090DF01C091F2020191C201F00001000C68
:10613000FF0E0201906FBB6F00011DDE015213E0E4
:1061400002018EC200F08F510F0B036E8EC291F2CE
:1061500003504009926FA66F8EC2A5F200012ADE9D
:10616000D4DF01C090F2FF0E0201BB6F000103DE1D
:10617000015203E1FF0E0201906F020190C201F093
:106180000001000C84C08FF283C08EF2D1DF01C009
:106190008CF2C00E02018C178B513F0B8C138AC2FC
:1061A0008DF284C09CF283C09BF2020E9E6F8C0E17
:1061B0009D6F010E9F6F0001DFDE86C09CF285C0DF
:1061C0009BF2020E02019E6F8D0E9D6F010E9F6F5E
:1061D0000001D2DE0FEF31F0BAEC03F08B86E7EC72
:1061E00006F0420E006E002EFED7000072A602D00E
:1061F00029EC07F0BAEC03F0E7EC06F08B9672B8E6
:1062000001D040DE72A406D00201986B976B0001AA
:10621000EEDE05D002018B6B8A6B0001B3D772A64C
:1062200002D029EC07F0BAEC03F0E7EC06F0FF0E21
:106230000201BB6F00019FDD015204E1FF0E016E00
:10624000026E10D0400E0201A66FA56B0001B2DDF8
:1062500001C088F2020102501F0B896F88C201F051
:1062600089C202F0000197EF34F0180E0201AC6F02
:106270009488FF0EBB6F00017EDD0201AE6BAD6B3B
:10628000AE510001905D0CE305E10201AD5100014A
:106290008F5D06E30201AD2BD8B4AE2BF1D7000120
:1062A0008B860201B06BAF6BB0510001905D10E3C3
:1062B00005E10201AF5100018F5D0AE3030E006E9C
:1062C000002EFED70201AF2BD8B4B02BEDD70001C2
:1062D00082B802D0D89001D0D8800201A837A9375F
:1062E000AA379498D890A437A537A63702E28B989E
:1062F00001D08B888B96B26BB16BB2510001905D6F
:1063000011E305E10201B15100018F5D0BE3110EB4
:10631000006E002EFED700D00201B12BD8B4B22BF4
:10632000ECD7000194880201AC07D8B402D0000178
:10633000B7D7A8C200F0A9C201F0AAC202F0ABC24E
:1063400003F00001000C0201A76BA00EA66FA56B65
:10635000A46B00018ADF1F0E0216036A000CF3DF34
:10636000000CBAEC03F0E7EC06F0210E006E002EF4
:10637000FED70201BB6B0001FEDC015202E18B86FD
:106380008B96FF0E0201BB6F0001F5DCE8DF03C056
:106390008BF202C08AF201C089F200C088F272DD7D
:1063A00088C200F089C201F08AC202F08BC203F0F9
:1063B000000C0201A76BA00EA66FA56BA46B0001D9
:1063C00054DF036A000CF5DF000CBAEC03F0E7ECD5
:1063D00006F0210E006E002EFED7FF0E0201BB6FED
:1063E0000001C9DCF0DF03C08BF202C08AF201C0F9
:1063F00089F200C088F246DD88C200F089C201F04F
:106400008AC202F08BC203F0ACEF34F072A409D060
:1064100084C08CF283C08BF2400E02018D6F08D0D5
:10642000000184C08CF283C08BF2400E02018D6F9C
:106430008CC28FF28BC28EF200017ADE01C08AF22A
:106440000201895303E08D518A1303D08D51FF0A55
:106450008A178CC29CF28BC29BF2020E9E6F8A0E30
:106460009D6F010E9F6F000187DD87EF34F00F0EE7
:1064700002018F6FD40E8E6F00015ADE01C08AF2C6
:106480000201895302E08A8D01D08A9D0F0E9C6F14
:10649000D40E9B6F020E9E6F8A0E9D6F010E9F6F32
:1064A00000016ADD87EF34F0020196C2A0F297C2C4
:1064B000A1F2080EA36BA3C2A7F2A66F97C2A5F222
:1064C00096C2A4F20001D1DE02019D5308E1A76B40
:1064D000090EA66FA56BA46B0001C7DE02019E6BBF
:1064E0009C519E5D35E29D5317E19BC203F09AC219
:1064F0009FF29BC2A0F2A76B090EA66FA56BA46BBF
:106500000001B3DEA0C2EAFF9FC2E9FF00C0EFFFB7
:1065100001C0ECFF15D002019BC203F09AC2E9FF53
:106520009BC2EAFFEFCFA0F2A16B0A0EA36BA3C23E
:10653000A7F2A66FA1C2A5F2A0C2A4F2000195DE47
:10654000020E02019A27000E9B23020E9E27C8D737
:106550000001000CD890020198339733963396C20D
:1065600000F097C201F098511F0B026E036A96C2A9
:10657000A0F297C2A1F20250D009A26F03C0A3F209
:1065800003C0A7F2A66F97C2A5F296C2A4F20001BB
:106590006CDE02019D5308E1A76BE00EA66FA56BB0
:1065A000A46B000162DE02019E6B9C519E5D35E290
:1065B0009D5317E19BC203F09AC29FF29BC2A0F2C7
:1065C000A76BE00EA66FA56BA46B00014EDEA0C208
:1065D000EAFF9FC2E9FF00C0EFFF01C0ECFF15D04A
:1065E00002019BC203F09AC2E9FF9BC2EAFFEFCF10
:1065F000A0F2A16BF00EA36BA3C2A7F2A66FA1C27B
:10660000A5F2A0C2A4F2000130DE020E02019A2718
:10661000000E9B23020E9E27C8D70001000C200EFF
:106620000201B46F9488FF0EBB6F0001BBEC2EF02B
:106630000201B66BB56BB6510001905D0CE305E14C
:106640000201B55100018F5D06E30201B52BD8B4FC
:10665000B62BF1D700018B860201B86BB76BB8512E
:106660000001905D10E305E10201B75100018F5D6B
:106670000AE3030E006E002EFED70201B72BD8B43A
:10668000B82BEDD7000182B802D0D89001D0D880C5
:106690000201B037B137B237B3379498D890AC37DE
:1066A000AD37AE37AF3702E28B9801D08B888B962F
:1066B000BA6BB96BBA510001905D11E305E10201BB
:1066C000B95100018F5D0BE3110E006E002EFED755
:1066D00000D00201B92BD8B4BA2BECD700019488B2
:1066E0000201B407D8B402D00001B5D7B0C200F09F
:1066F000B1C201F0B2C202F0B3C203F00001000C5B
:1067000002019651FE0B006E97C201F098C202F092
:10671000036AA46F97C2A5F298C2A6F20350C009FB
:10672000A76FAF6F98C2AEF297C2ADF200C0ACF2E5
:10673000000175DF02019D5310E1C10EAF6FAE6B1A
:10674000AD6BAC6B00016BDF03C0A2F202C0A1F223
:1067500001C0A0F200C09FF202019E6B9C519E5DA1
:1067600063E29D5332E1C10EAF6FAE6BAD6BAC6BAC
:10677000000155DF03C0A2F202C0A1F201C0A0F2E5
:1067800000C09FF202019BC203F09A519A2BD8B429
:106790009B2BE96E03C0EAFF9FC2EFFF9BC203F091
:1067A0009A519A2BD8B49B2BE96E03C0EAFFA0C282
:1067B000EFFF9BC203F09A519A2BD8B49B2BE96E42
:1067C00003C0EAFFA1C2EFFF2CD09BC203F09AC224
:1067D000E9FF9BC2EAFFEFCFA4F2ECCFA5F2ECCF2A
:1067E000A6F2ECCFA7F2A4C200F0A5C201F0A6C2A7
:1067F00002F0036AA4C2A8F2A5C2A9F2A6C2AAF234
:106800000350C209AB6FAF6FA6C2AEF2A5C2ADF224
:10681000A4C2ACF2000103DF030E02019A27000EAE
:106820009B23030E9E279AD70001000C000CD890E2
:106830004E34036AF2CF96F2F29E24EC02F0090085
:10684000F5CF03F0020196BFF28E00018D6F03C0F9
:106850008EF0EA6A8D0EE96E91C299F290C298F2BA
:106860008FC297F28EC296F293C29BF292C29AF2B4
:1068700094C29CF295C29DF235EC02F0000C02012C
:106880008A6B8B6B8C6B8D6B916BFD0E906F8F6B2E
:10689000360E8E6F020E936F8A0E926F030E946FF8
:1068A000956B0001C4DF0201895302E08A8104D0A4
:1068B0008A918B6B8C6B8D6B916BFD0E906F8F6BD8
:1068C000360E8E6F020E936F8A0E926F030E946FC8
:1068D000010E956F0001ABDF87EF34F00201886B8A
:1068E000000193A104D0010E0201886F00014E50F7
:1068F00005E0010A06E0030A07E009D088C289F230
:1069000085D588C289F2B3D588C289F2B8D7B8EFE5
:1069100034F0FC0E936F050E906F940E8F6F4E50F7
:1069200005E0010A0DE0030A16E01FD055D402016C
:10693000876B866B02C085F201C084F2000115D01E
:1069400010DD0FDD03C087F202C086F201C085F2C0
:1069500000C084F20AD039D503C087F202C086F2A3
:1069600001C085F200C084F200D083C293F0B6D794
:1069700042EC2FF0FF0E0201BB6F0001BBEC2EF0CA
:10698000015207E10201876BFF0E866F856F846FEE
:10699000000184C200F085C201F086C202F087C205
:1069A00003F0E3EF34F0030E0201826F020E816FF9
:1069B0007C0E806F0A50020802E181C182F282C21D
:1069C00083F20001A6D703C07FF202C07EF201C0AD
:1069D0007DF200C07CF2D00E0101806F0201BB6B22
:1069E0000001BBEC2EF0015202E0000E01D0010EBE
:1069F0000101816F020181C203F08051802BD8B464
:106A0000812BE96E03C0EAFFEFCF82F101010201A1
:106A100081C203F08051802BD8B4812BE96E03C072
:106A2000EAFFEFCF83F1010180C2E9FF81C2EAFFF3
:106A3000EFCF84F10101050E0A6E000191EC02F026
:106A400037EF3FF0400E0201A66FA56B0001DAECB4
:106A50002EF002C003F001C000F01F0E031601C0AB
:106A600001F003C002F0000CEDDF025054EF35F0EE
:106A70000201856BFF0E846F836F826FBB6B000119
:106A8000BBEC2EF0015237E18B86640E0201BD6F24
:106A9000000106EC05F08B964E5005E0010A0DE072
:106AA000030A15E01ED0E0D70201856B846B02C09B
:106AB00083F201C082F2000114D051DC03C085F2E0
:106AC00002C084F201C083F200C082F20AD07BDCF3
:106AD00003C085F202C084F201C083F200C082F2DA
:106AE00000D0FF0E0201BB6F0001BBEC2EF093A3A0
:106AF00002D042EC2FF082C200F083C201F084C2C7
:106B000002F085C203F08CEF35F0020E0201816FB6
:106B10007C0E806F0001ACD703C07FF202C07EF212
:106B200001C07DF200C07CF2D00E0101806F020135
:106B3000BB6B0001BBEC2EF0015202E0000E01D055
:106B4000010E0101816F020181C203F08051802B8F
:106B5000D8B4812BE96E03C0EAFFEFCF82F10101C7
:106B6000020181C203F08051802BD8B4812BE96EE1
:106B700003C0EAFFEFCF83F1010180C2E9FF81C2C8
:106B8000EAFFEFCF84F10101050E0A6E000191ECDE
:106B900002F037EF3FF093A102D00201978D84C03D
:106BA0009CF283C09BF2020E02019E6F970E9D6FB6
:106BB000010E9F6F0001BCEC2FF0800E0201A66F4A
:106BC000A56B0001DAEC2EF0000C96C298F295C28B
:106BD00097F2F7EC2FF00201976B0001DCDF19EF61
:106BE00036F002019A8F000193A103D002019A8D21
:106BF00000019AC2A6F299C2A5F2DAEC2EF0000CBE
:106C0000020195C297F296511F0B986F9A6F95C229
:106C100099F20001E6DF19EF36F072A405D094C2B4
:106C200096F293C295F2D1D794C296F293C295F29E
:106C3000E7D703EF38F0020191C200F092C201F0F1
:106C400093511F0B026E036A91C296F292C297F2A1
:106C500002508009986F03C099F203C0A7F2A66F93
:106C600092C2A5F291C2A4F2000135EC31F003EF1B
:106C700038F0FF0E0201956F966F976F986B010EBB
:106C8000A66FA56B0001DAEC2EF003EF38F0FF0ED3
:106C90000201916F926F936F946BBB6B0001BBEC21
:106CA0002EF0015231E093A304D0050E906F940EA4
:106CB0008F6F4E5005E0010A0DE0030A16E020D068
:106CC000C1DE0201946B936B02C092F201C091F29B
:106CD000000116D0A3EC31F003C094F202C093F28D
:106CE00001C092F200C091F20BD0D9EC31F003C098
:106CF00094F202C093F201C092F200C091F200D06F
:106D000093A302D042EC2FF091C200F092C201F0A6
:106D100093C202F094C203F0000C82B0FED7080EBA
:106D2000006E02019A6B008E0ED0009E0CD0D8909F
:106D300082B0D8809A33008C06D0009C002EF7D702
:106D40009AC201F016D0050EE96E000E00BE550E77
:106D5000016E012EFED7E92EF8D75C0E00BE190E8B
:106D6000016E012EFED7000000BEDFD700BCE5D7C4
:106D7000DED70001DAEF36F0020195819593948019
:106D80003CA207D093C2E9FF94C2EAFF010EEF6E66
:106D900035D095B333D0040082B015D094C203F03F
:106DA00093C2E9FF94C2EAFFEACF99F2E9CF98F2E1
:106DB0000001B3D799C2EAFF98C2E9FF01C0EFFF13
:106DC0000201958319D000018EEC05F001520AE012
:106DD00068EC02F00150020804E1020195839591EC
:106DE00000010AD00201BB6B0001BBEC2EF0015286
:106DF00003E00201958395910201CBD7000E95B176
:106E0000010E016E0001A9EF37F0020194519EA816
:106E1000FED7AD6E0001000C080E0201946F000158
:106E2000F4DF93C294F2F1DF000C02019581959397
:106E300095B345D0BB6B0001BBEC2EF00152D8B42A
:106E400002D002013CD08EEC05F0015236E094C233
:106E500003F093C296F294C297F2000168EC02F03C
:106E600097C2EAFF96C2E9FF01C0EFFF94C203F0A8
:106E7000020193C2E9FF94C2EAFFEF50080812E151
:106E800094C203F093C296F294C297F2000168ECA8
:106E900002F097C2EAFF96C2E9FF01C0EFFF0201CC
:106EA00095830BD094C203F093C2E9FF94C2EAFF2A
:106EB000EF50020802E1958395910201B9D7000EC7
:106EC00095B1010E016E0001BDEF37F08B90080EF9
:106ED000016E00D00000018E10D0019E020194339B
:106EE0000001D8B08B80D8A08B90018C06D0019C7B
:106EF000012EF4D700D000008B80050E006EE96AE9
:106F0000E92EFED7002EFBD7610EE96EE92EFED7E3
:106F100000D001BEE2D701BCEAD793EF37F09490DE
:106F200093C294F2D3D7C3EF37F00201919191B19C
:106F300039D0BB6B0001BBEC2EF00152D8B402D0AB
:106F4000020130D0020E0201946F920E936F000185
:106F500013D7015223E002019251010A000101E01E
:106F600018D0010E0201936F000156DF020E0201DC
:106F7000946F920E936F000158D7015205E03C9236
:106F800092C293F2CCD704D03C82020191810001DD
:106F900004D092C293F240DF00D002D0020191816E
:106FA0000201C5D7000111EF38F0FF0E02018D6F0D
:106FB0008E6F8F6F906BBB6B0001BBEC2EF001529C
:106FC00022E04E5005E0010A0CE0030A13E01BD05A
:106FD00089C292F288C291F289C294F288C293F275
:106FE0001CD68BC294F28AC293F289C292F288C2F2
:106FF00091F221D68BC294F28AC293F289C292F2A4
:1070000088C291F236D643DE03C090F202C08FF2FE
:1070100001C08EF200C08DF202018C5303E000012A
:1070200084D702018DC200F08EC201F08FC202F03F
:1070300090C203F0000146EF38F002018281020E97
:10704000816F7C0E806F0A50050809E18291010171
:107050008451010B016EE8A003D00201828101017D
:107060000201866B83C185F282C184F281C183F201
:10707000000E82B1010E86C28BF283C18AF282C1F8
:1070800089F281C188F28C6F00018FD703C07FF233
:1070900002C07EF201C07DF200C07CF2D00E010180
:1070A000806F0201BB6B0001BBEC2EF0015202E0CD
:1070B000000E01D0010E0101816F020181C203F0B7
:1070C0008051802BD8B4812BE96E03C0EAFFEFCF4B
:1070D00082F10101020181C203F08051802BD8B4FA
:1070E000812BE96E03C0EAFFEFCF83F1010180C27B
:1070F000E9FF81C2EAFFEFCF84F10101050E0A6EBC
:10710000000191EC02F037EF3FF0200E0201976F83
:10711000000141DD99EF38F03F0E02019A6FFF0E3A
:10712000996F00015EDD99EF38F072A401D0EDD7C0
:10713000F3D7CDEF38F00201A76BC00EA66FA56B99
:10714000A46B000135EC31F0640E0201BD6F00014B
:1071500006EC05F0CDEF38F0020E0201A66FA56B2C
:107160000001DAEC2EF0640E0201BD6F000106ECA6
:1071700005F0CDEF38F0FF0E0201BB6F0001BBEC54
:107180002EF001520AE04E5005E0010A04E0030A25
:1071900003E003D0CAD7CFD7DFD7FF0E0201BB6F02
:1071A0000001BBEC2EF0015208E10201856BFF0EDD
:1071B000846F836F826F0BD0000169DD03C085F29D
:1071C00002C084F201C083F200C082F2020182C2D6
:1071D00000F083C201F084C202F085C203F0000116
:1071E000F9EF38F0020E0201816F7C0E806F000112
:1071F000C2D703C07FF202C07EF201C07DF200C0A0
:107200007CF2D00E0101806F0201BB6B0001BBEC70
:107210002EF0015202E0000E01D0010E0101816F3B
:10722000020181C203F08051802BD8B4812BE96E1A
:1072300003C0EAFFEFCF82F10101020181C203F036
:107240008051802BD8B4812BE96E03C0EAFFEFCFC9
:1072500083F1010180C2E9FF81C2EAFFEFCF84F12F
:107260000101050E0A6E000191EC02F037EF3FF0CC
:10727000020E0201816F7C0E806F000108DD03C0E9
:107280007FF202C07EF201C07DF200C07CF2D00E1F
:107290000101806F0201BB6B0001BBEC2EF00152BB
:1072A00002E0000E01D0010E0101816F020181C2D6
:1072B00003F08051802BD8B4812BE96E03C0EAFF24
:1072C000EFCF82F10101020181C203F08051802BD6
:1072D000D8B4812BE96E03C0EAFFEFCF83F101013F
:1072E00080C2E9FF81C2EAFFEFCF84F10101050E00
:1072F0000A6E000191EC02F037EF3FF0030E02013D
:107300008A6F000159EC02F084C28AF259EC02F053
:1073100084C279F2000C80C18AF259EC02F00101BA
:1073200080510201791B0001000C02018D6B8E6BF4
:10733000FF0EBB6F0001BBEC2EF001520AE0020110
:10734000A66BA56B0001DAEC2EF002C08EF201C034
:107350008DF202018DC201F08EC202F00001000C1C
:10736000FF0E02018B6F8C6FBB6F0001BBEC2EF028
:10737000015216E0020189C28EF28AC28FF2800E9B
:10738000916B91C2A7F2A66F8AC2A5F289C2A4F23C
:10739000000135EC31F0C9DF02C08CF201C08BF284
:1073A000FF0E0201BB6F0001BBEC2EF0015204E1A5
:1073B000FF0E02018C6F8B6F02018BC201F08CC239
:1073C00002F0000129EF3AF079C28AF259EC02F09A
:1073D00068EC02F001500608FBE1000C010E02010E
:1073E000806F800E7F6F82C17EF281C17DF283C18A
:1073F00082F2030E8225836F846F00017FDF02011A
:107400007FC2E9FF80C2EAFFE00EEF6E000183DF7A
:1074100002017FC2E9FF80C2EAFF81C1EFFF0001E4
:107420007ADF02017FC2E9FF80C2EAFF82C1EFFF7B
:10743000000171DF02017C532DE07EC284F27DC227
:1074400083F282C285F284C28AF283C289F2000189
:1074500087D702C088F201C087F287C280F15BDF64
:1074600088C280F158DF020E0201866F8551865D69
:1074700010E200015ADF02C088F201C087F287C221
:1074800080F149DF88C280F146DF020E02018627C3
:10749000EDD71FD07EC284F27DC283F282C285F214
:1074A00084C28FF283C28EF2000198EC30F001C0EA
:1074B00080F131DF010E0201866F8551865D09E2A0
:1074C000000185EC30F001C080F125DF0201862B40
:1074D000F4D7000179DF000C020185C28CF286C26C
:1074E0008DF2810E8F6B8FC2A7F2A66F86C2A5F2B6
:1074F00085C2A4F2000135EC31F002018A6B89519A
:107500008A5D2CE2FF0EBB6F0001BBEC2EF0015236
:107510001DE0020187C2E9FF88C2EAFFECCF03F059
:10752000ED52EFCF8CF203C08DF2820E8F6B8FC2C3
:10753000A7F2A66F03C0A5F28CC2A4F2000135EC3D
:1075400031F093A302D042EC2FF000D0020E0201E2
:107550008727D8B0882B020E8A27D1D70001E5EF04
:107560003AF0FF0E0201BB6F0001BBEC2EF001529E
:107570002CE04E5005E0010A10E0030A1BE025D084
:1075800081C29CF280C29BF283C29EF282C29DF2B3
:1075900084C29FF2BCEC2FF018D081C29CF280C252
:1075A0009BF283C29EF282C29DF284C29FF2BCEC27
:1075B0002FF00BD081C286F280C285F283C288F29E
:1075C00082C287F284C289F287D7FBEF3AF082C188
:1075D0007EF281C17DF2030E0A5C02017F6F7EC2E2
:1075E00081F27DC280F2010E836F830E826F7FC2B3
:1075F00084F20001B6D7070E0101806F010E0A6EFA
:10760000000191EC02F037EF3FF002018DC290F2E1
:107610008EC291F2830E936B93C2A7F2A66F8EC2B5
:10762000A5F28DC2A4F2000135EC31F0030E020187
:10763000A66FA56B0001DAEC2EF00250000C0201DF
:107640008B6B8C6BFF0EBB6F0001BBEC2EF00152FD
:107650000EE04E50020A01E00AD08AC28EF289C2C0
:107660008DF2D3DF02C08CF201C08BF200D0020198
:107670008BC201F08CC202F00001D2EF3BF002019C
:107680008CC28DF2200EA66F8CC2A5F20001DAEC3E
:107690002EF0400E0201A66FA56B0001DAEC2EF071
:1076A00001C08DF202010250036A016E0001000C5C
:1076B00002018CC200F08D51030B036E8CC28EF25E
:1076C000035020098F6FA66F8CC2A5F20001DAEC7F
:1076D0002EF0020E0201926F000121EC30F00150F9
:1076E000000C02018B6BFF0EBB6F0001BBEC2EF098
:1076F000015213E04E5003E0010A07E00ED089C2A8
:107700008CF2BDDF01C08BF208D08AC28DF289C233
:107710008CF2CEDF01C08BF200D002018BC201F0EF
:107720000001FDEF3BF0010E0201806F800E7F6FC4
:1077300082C17EF281C17DF283C182F2030E822575
:10774000836F846F0001DADD02017FC2E9FF80C22E
:10775000EAFFE20EEF6E0001DEDD02017FC2E9FF0B
:1077600080C2EAFF81C1EFFF0001D5DD02017FC2C7
:10777000E9FF80C2EAFF82C1EFFF0001CCDD020118
:107780007C5323E07EC284F27DC283F282C285F202
:10779000866B8551865D18E284C28AF283C289F2C3
:1077A00000014DD702C088F201C087F287C280F184
:1077B000B2DD88C280F1AFDD020E02018327000E28
:1077C0008423020E8627E5D71ED07EC284F27DC2B6
:1077D00083F282C285F2866B8551865D14E284C293
:1077E00003F08351832BD8B4842B876F03C088F2B6
:1077F00003C08AF2896F000174D701C080F18BDD6C
:107800000201862BE9D70001DFDD000CFF0E02012B
:10781000BB6F0001BBEC2EF001520AE002018BC2EB
:107820008CF2300EA66F8BC2A5F20001DAEC2EF0BE
:10783000000C0201886B8751885D17E2885184250E
:10784000896F8C6F00011BDF036A02018851852557
:10785000E96E86510320EA6EEFCF89F289C28BF27E
:107860000001D4DF0201882BE6D70001B6EF3CF01F
:107870000201896B8851895D1CE2895184258A6FD8
:10788000000E85218B6F8D6F8AC28CF2000110DF94
:10789000036A020189518625E96E87510320EA6E49
:1078A000EFCF8AF28AC28BF20001B0DF0201892B8E
:1078B000E1D70001B6EF3CF085C28EF284C28DF2B2
:1078C000A4DE0201896B8851895D1FE286C2E9FF4F
:1078D00087C2EAFFECCF03F0ED52EFCF8BF203C08B
:1078E0008CF2850E8E6B8EC2A7F2A66F03C0A5F236
:1078F0008BC2A4F2000135EC31F0020E02018627A2
:10790000D8B0872B020E8927DED70001B6EF3CF0F6
:10791000FF0E0201BB6F0001BBEC2EF0015226E00E
:107920004E5005E0010A0CE0030A15E01FD07FC2AB
:1079300084F282C286F281C285F283C287F279D74D
:1079400080C285F27FC284F282C287F281C286F24F
:1079500083C288F28DD780C285F27FC284F282C250
:1079600087F281C286F283C288F2A6D7CCEF3CF0C0
:1079700082C17DF281C17CF2030E0A5C02017E6F3E
:107980007DC280F27CC27FF2010E826F830E816F16
:107990007EC283F20001BCD7070E0101806F010E89
:1079A0000A6E000191EC02F037EF3FF00201806BAC
:1079B00083C17FF282C17EF281C17DF284C10AF06F
:1079C00080C291F27FC290F27EC28FF27DC28EF2AF
:1079D000010E936F840E926F0AC094F2956B0001B2
:1079E00017EC34F0C40E0101806F040E0A2600016A
:1079F00091EC02F037EF3FF00201806B83C17FF220
:107A000082C17EF281C17DF2040E0A5C816F80C268
:107A100091F27FC290F27EC28FF27DC28EF2010E91
:107A2000936F840E926F81C294F2010E956F0001E4
:107A300017EC34F0070E0101806F010E0A6E000191
:107A400091EC02F037EF3FF0010E02017F6F810EE3
:107A50007FC27DF27C6F970E0101806F7DC203F0C3
:107A60007CC27EF27DC27FF2000142EC2FF07FC229
:107A7000EAFF7EC2E9FF02C0ECFFED5201C0EFFF5A
:107A8000030E0A6E91EC02F037EF3FF00F0E020189
:107A90008F6FFC0E8E6F000198EC30F001C089F200
:107AA0000F0E02019C6FFC0E9B6F020E9E6F850EE7
:107AB0009D6F010E9F6F0001BCEC2FF002018A6BDD
:107AC00088518A5D54E2036A8A518625016E875186
:107AD000032201C08BF203C08CF20F0E8F6FFD0EDC
:107AE0008E6F000198EC30F08CC2EAFF8BC2E9FF88
:107AF00001C0EFFF010E02018A25036A8625016E8F
:107B00008751032201C08CF203C08DF2000185EC85
:107B100030F08DC2EAFF8CC2E9FF01C0EFFF020E18
:107B200002018A25036A8625016E8751032201C05E
:107B30008CF203C08DF2000185EC30F08DC2EAFFBB
:107B40008CC2E9FF01C0EFFF0201852B0F0E9C6F75
:107B5000FC0E9B6F020E9E6F850E9D6F010E9F6F38
:107B60000001BCEC2FF0030E02018A27A9D70F0EEB
:107B70009C6FFC0E9B6F020E9E6F890E9D6F010E17
:107B80009F6F0001BCEC2FF0DBEF3DF0FF0E020118
:107B9000BB6F0001BBEC2EF001520DE04E50010A0C
:107BA00001E009D080C285F283C287F282C286F2E8
:107BB00084C288F26BD7FDEF3DF0010E02017F6FAA
:107BC000810E7FC27DF27C6F83C10AF07DC203F01B
:107BD0007CC2E9FF7DC2EAFFECCF7FF2ED52EFCF2E
:107BE0007EF27FC281F27EC280F2010E836F830E2D
:107BF000826F0AC084F20001C9D7E60E0101806FCE
:107C0000030E0A26000191EC02F037EF3FF00F0E51
:107C100002018F6FFC0E8E6F000198EC30F001C0F6
:107C20008AF202018B6B89518B5D53E20F0E9C6FC0
:107C3000FC0E9B6F020E9E6F860E9D6F010E9F6F56
:107C40000001BCEC2FF0036A02018B5187258C6F79
:107C5000885103208D6F0F0E9C6FFD0E9B6F8DC2A0
:107C60009EF28CC29DF2010E9F6F0001BCEC2FF0C2
:107C7000010E02018B25036A87258D6F8851032031
:107C80008E6F0F0E9C6FFE0E9B6F8EC29EF28DC28A
:107C90009DF2010E9F6F0001BCEC2FF0020E02015D
:107CA0008B25036A87258D6F885103208E6F0F0EF9
:107CB0009C6FFF0E9B6F8EC29EF28DC29DF2010ED5
:107CC0009F6F0001BCEC2FF00201862B030E8B2767
:107CD000AAD70F0E9C6FFC0E9B6F020E9E6F8A0E32
:107CE0009D6F010E9F6F0001BCEC2FF08DEF3EF0F9
:107CF000FF0E0201BB6F0001BBEC2EF001520DE044
:107D00004E50010A01E009D081C286F284C288F295
:107D100083C287F285C289F27AD7B0EF3EF0010EB6
:107D200002017F6F810E7FC27DF27C6F7DC203F006
:107D30007CC2E9FF7DC2EAFFECCF7FF2ED52EFCFCC
:107D40007EF2030E0A5C806F7FC282F27EC281F2F5
:107D5000010E846F830E836F80C285F20001C8D745
:107D6000070E0101806F010E0A6E000191EC02F016
:107D700037EF3FF080C181F1FF0E0101806F020EED
:107D80000A6E000191EC02F037EF3FF002017B53E5
:107D900001E06ED001018051520803E10001D3EFF0
:107DA00034F08051530803E1000185EF35F0805134
:107DB000540803E100011DEF38F08051550803E13C
:107DC0000001F2EF38F08051560803E1000138EF6E
:107DD00039F08051600807E102017C6B0001EEEC94
:107DE00039F045D001018051690808E1010E020116
:107DF0007C6F0001EEEC39F03AD00101805161084E
:107E000003E10001E7EF3AF08051620806E1020168
:107E10007C6B000188DC2BD0010180516A0807E1EE
:107E2000010E02017C6F00017EDC21D00101805136
:107E3000630802E100019CD58051650802E1000160
:107E4000B5D58051640802E10001D6D5805166089D
:107E500002E10001F9D58051670802E10001ADD6C9
:107E60008051680802E100015AD7000183D702015E
:107E70000001CCEF3FF0F86AD09E0E8EEA6AE96A04
:107E8000810EAF6EA60EAC6E900EAB6E810EAF6E15
:107E9000A60EAC6E900EAB6E810EAF6EA60EAC6EE3
:107EA000900EAB6E810EAF6EA60EAC6E900EAB6EEA
:107EB000810EAF6EA60EAC6E900EAB6E8B808B807B
:107EC000C180C182C184C196056A066A940E8F6F13
:107ED000050E906F3C92040E946FFF0E956F966F97
:107EE000976B986F996F9A6B9B6F9C6F9D6B9E6F52
:107EF0009F6FA06BA16FA26BA36BA46FA56BA66B0A
:107F0000A76FA86BA96BAA6FAB6BAC6BAD6FAE6BB9
:107F1000AF6BB06FB16BB26BB36FB46BB56BB66F69
:107F2000B76BB86BB96FBA6BBB6BBC6FBD6BBE6B1D
:107F3000BF6FC06BC16BC26FC36BC46BC56FC66BC9
:107F4000C76BC86FC96BCA6BCB6FCC6BCD6BCE6F79
:107F5000CF6BD06B010ED16F49EF02F0830ED56E5F
:107F6000D76AD66AF19AF28AC00EF212D180E6EC94
:107F700002F0D16B928693948A84066A04004BEFD8
:107F800004F001C07AF27AC27BF248EF2EF001C011
:107F90007AF27AC27BF2FAD6F1D70300FFFFFFFF35
:107FA000FFFFFFFFFFFFFFFFFFFFFFFFFFFFFFFFE1
:107FB000FFFFFFFFFFFFFFFFFFFFFFFFFFFFFFFFD1
:107FC000FFFFFFFFFFFFFFFFFFFFFFFFFFFFFFFFC1
:107FD000FFFFFFFFFFFFFFFFFFFFFFFFFFFFFFFFB1
:107FE000FFFFFFFFFFFFFFFFFFFFFFFFFFFFFFFFA1
:107FF000FFFFFFFFFFFFFFFFFFFFFFFFFFFFFFFF91
:0200000400F00A
:10000000FFFFFFFFFFFFFFFFFFFFFFFFFFFFFFFF00
:10001000FFFFFFFFFFFFFFFFFFFFFFFFFFFFFFFFF0
:10002000FFFFFFFFFFFFFFFFFFFFFFFFFFFFFFFFE0
:10003000FFFFFFFFFFFFFFFFFFFFFFFFFFFFFFFFD0
:10004000FFFFFFFFFFFFFFFFFFFFFFFFFFFFFFFFC0
:10005000FFFFFFFFFFFFFFFFFFFFFFFFFFFFFFFFB0
:10006000FFFFFFFFFFFFFFFFFFFFFFFFFFFFFFFFA0
:10007000FFFFFFFFFFFFFFFFFFFFFFFFFFFFFFFF90
:10008000FFFFFFFFFFFFFFFFFFFFFFFFFFFFFFFF80
:10009000FFFFFFFFFFFFFFFFFFFFFFFFFFFFFFFF70
:1000A000FFFFFFFFFFFFFFFFFFFFFFFFFFFFFFFF60
:1000B000FFFFFFFFFFFFFFFFFFFFFFFFFFFFFFFF50
:1000C000FFFFFFFFFFFFFFFFFFFFFFFFFFFFFFFF40
:1000D000FFFFFFFFFFFFFFFFFFFFFFFFFFFFFFFF30
:1000E000FFFFFFFFFFFFFFFFFFFFFFFFFFFFFFFF20
:1000F000FFFFFFFFFFFFFFFFFFFFFFFFFFFFFFFF10
:020000040030CA
:0E00000000260E0F000181000FC00F800F4080
:020000040020DA
:08000000FFFFFFFFFFFFFFFF00
:00000001FF
